:0400000076EF00F0A7
:060008004D82F9EF42F009
:100018004D80D8CFC7F0E8CFC8F0E0CFC9F0FACF0D
:10002800CAF0FBCFCBF0E9CFCCF0EACFCDF0E1CFEF
:10003800CEF0E2CFCFF0D9CFD0F0DACFD1F0F3CFF6
:10004800D2F0F4CFD3F0F6CFD4F0F7CFD5F0F8CF85
:10005800D6F0F5CFD7F04DC0D8F04EC0D9F04FC08C
:10006800DAF050C0DBF09DAC3CEF00F03EEF00F062
:100078004AEF00F09EAC43EF00F045EF00F04AEF86
:1000880000F0010E4B6E9E9C4AEF00F0DBC050F072
:10009800DAC04FF0D9C04EF0D8C04DF0D7C0F5FF48
:1000A800D6C0F8FFD5C0F7FFD4C0F6FFD3C0F4FF21
:1000B800D2C0F3FFD1C0DAFFD0C0D9FFCFC0E2FF72
:1000C800CEC0E1FFCDC0EAFFCCC0E9FFCBC0FBFF4B
:1000D800CAC0FAFFC9C0E0FFC8C0E8FFC7C0D8FF60
:1000E8004D90100059EF48F03C50D8B47EEF00F026
:1000F80080EF00F04DEF18F003EC4DF00401826F33
:1001080024EF18F003EC4DF00401896F96EF00F02E
:10011800010E3B6E4DEF18F0000E3B6E4DEF18F0E0
:100128004DEF18F08951300AD8B48CEF00F0010A6D
:10013800D8B490EF00F04DEF18F04DEF18F04DEFF8
:1001480018F0BBEC4DF0A9C013F0146A000E166E3F
:100158000A0E156E7BEC45F01350150F0401916FD4
:10016800320E1F6EEF0E206E91C421F0CBEC4EF0D4
:10017800A9C013F0146A000E166E0A0E156E61EC13
:1001880046F01350150F0401926F7F0E1F6EEF0E8D
:10019800206E92C421F0CBEC4EF0AAC013F0146A82
:1001A800000E166E0A0E156E7BEC45F01350150FF7
:1001B8000401916F480E1F6EEF0E206E91C421F05E
:1001C800CBEC4EF0AAC013F0146A000E166E0A0E9D
:1001D800156E61EC46F01350150F0401926F950EE1
:1001E8001F6EEF0E206E92C421F0CBEC4EF04DEF57
:1001F80018F0BBEC4DF0A9C013F0146A000E166E8F
:100208000A0E156E7BEC45F01350150F0401916F23
:100218003D0E1F6EEF0E206E91C421F0CBEC4EF018
:10022800A9C013F0146A000E166E0A0E156E61EC62
:1002380046F01350150F0401926F8A0E1F6EEF0ED1
:10024800206E92C421F0CBEC4EF0AAC013F0146AD1
:10025800000E166E0A0E156E7BEC45F01350150F46
:100268000401916F530E1F6EEF0E206E91C421F0A2
:10027800CBEC4EF0AAC013F0146A000E166E0A0EEC
:10028800156E61EC46F01350150F0401926FA00E25
:100298001F6EEF0E206E92C421F0CBEC4EF0A8C07A
:1002A80013F0146A000E166E0A0E156E7BEC45F0FC
:1002B8001350150F0401916F270E1F6EEF0E206E5D
:1002C80091C421F0CBEC4EF0A8C013F0146A000ED4
:1002D800166E0A0E156E61EC46F01350150F0401E8
:1002E800926F740E1F6EEF0E206E92C421F0CBEC4D
:1002F8004EF0A7C013F0146A000E166E0A0E156EA3
:100308007BEC45F01350150F0401916F5E0E1F6EC4
:10031800EF0E206E91C421F0CBEC4EF0A7C013F085
:10032800146A000E166E0A0E156E61EC46F0135034
:10033800150F0401926FAB0E1F6EEF0E206E92C464
:1003480021F0CBEC4EF0A6C013F0146A000E166E26
:100358000A0E156E7BEC45F01350150F0401916FD2
:10036800690E1F6EEF0E206E91C421F0CBEC4EF09B
:10037800A6C013F0146A000E166E0A0E156E61EC14
:1003880046F01350150F0401926FB60E1F6EEF0E54
:10039800206E92C421F0CBEC4EF04DEF18F003EC38
:1003A8004DF00401836F03EC4DF00401846F03ECFE
:1003B8004DF00401856F03EC4DF00401866F03ECEA
:1003C8004DF00401876F03EC4DF00401886F03ECD6
:1003D8004DF00401886F03EC4DF00401886F84C46C
:1003E800DCF085C4DDF086C4DEF087C4DFF088C4A5
:1003F800E0F0835171EC4BF04DEF18F04DEF18F031
:100408004DEF18F0B2C0B0F0B3C0B1F00001B15177
:1004180009E1FB0EB05DD8A014EF02F016EF02F070
:100428003EEF02F0F20EB025B06FFE0EB121B16FB3
:10043800000EDF6F380EE06F410EE16FB0C01BF0A9
:10044800B1C01CF00CEC50F01BC0DCF01CC0DDF09F
:100458001DC0DEF0AEEC43F0DCC0F5F2DDC0F6F214
:10046800DEC0F7F242EC42F0F5C2B0F0F6C2B1F0ED
:1004780045EF02F0000E0001B16F000EB06F45EFBE
:1004880002F00001AF5109E1C90EAE5DD8A04FEFEF
:1004980002F051EF02F07CEF02F0E90EAE5D030EC0
:1004A800AF59D8A05AEF02F05CEF02F062EF02F009
:1004B800030EAF6FE80EAE6F62EF02F0380EAE2596
:1004C800AE6FFF0EAF21AF6FAEC0F4F3AFC0F5F360
:1004D8000301D890F533F433D890F533F433D8903A
:1004E800F533F433F4C3AEF0F5C3AFF083EF02F0A5
:1004F800000E0001AF6F000EAE6F83EF02F0B0C0C8
:10050800C6F05C0E1F6EEC0E206EB0C021F0CBEC76
:100518004EF0000E1F6EEF0E206E0001B051080F56
:10052800216ECBEC4EF0F20E1F6EEE0E206E000127
:10053800B051060F216ECBEC4EF0E40E1F6EEE0E9E
:10054800206E0001B051040F216ECBEC4EF0D60E98
:100558001F6EEE0E206E0001B051020F216ECBEC23
:100568004EF0C80E1F6EEE0E206EB0C021F0CBEC20
:100578004EF0BA0E1F6EEE0E206E0001B051FE0F47
:10058800216ECBEC4EF0AC0E1F6EEE0E206E00010D
:10059800B051FC0F216ECBEC4EF09E0E1F6EEE0E8E
:1005A800206E0001B051FA0F216ECBEC4EF0900E88
:1005B8001F6EEE0E206E0001B051F80F216ECBECCD
:1005C8004EF00E0E1F6EEE0E206E050E216ECBEC59
:1005D8004EF0830E1F6EEC0E206EAEC021F0CBECF9
:1005E8004EF00001C651C25DD8B0FDEF02F0FFEF3A
:1005F80002F00FEF03F0B905D8A405EF03F007EFF9
:1006080003F00FEF03F0000EB96FF1EC45F00FEFB8
:1006180003F00FEF03F00001C051C65DD8B017EF2B
:1006280003F019EF03F04DEF18F0B905D8A41FEF48
:1006380003F021EF03F04DEF18F0000EB96FF1EC65
:1006480045F04DEF18F04DEF18F04DEF18F003ECB2
:100658004DF00401896FBBEF17F0FF004DEF18F064
:100668002DEC2EF04DEF18F0F00E136E000E146EF8
:10067800000E80EC4FF04DEF18F0C1EC34F04DEF68
:1006880018F003EC4DF00001946F03EC4DF00001FD
:10069800956F03EC4DF00001966F03EC4DF00001EF
:1006A800986F03EC4DF00001976F03EC4DF00001DB
:1006B800996FC00E136E010E146E38EC47F04DEFB3
:1006C80018F003EC4DF00001946F03EC4DF00001BD
:1006D800956F03EC4DF00001966F03EC4DF00001AF
:1006E800986F03EC4DF00001976F03EC4DF000019B
:1006F800996F900E136E010E146E38EC47F04DEFA3
:1007080018F003EC4DF00001946F03EC4DF000017C
:10071800956F03EC4DF00001966F03EC4DF000016E
:10072800986F03EC4DF00001976F03EC4DF000015A
:10073800996F600E136E010E146E38EC47F04DEF92
:1007480018F003EC4DF00001956F03EC4DF000013B
:10075800966F03EC4DF00001986F03EC4DF000012B
:10076800976F03EC4DF00001996F900E136E020E17
:10077800146E38EC47F04DEF18F003EC4DF0000123
:10078800956F03EC4DF00001966F03EC4DF00001FE
:10079800986F03EC4DF00001976F03EC4DF00001EA
:1007A800996F600E136E020E146E38EC47F04DEF21
:1007B80018F003EC4DF00001956F03EC4DF00001CB
:1007C800966F03EC4DF00001986F03EC4DF00001BB
:1007D800976F03EC4DF00001996F300E136E010E08
:1007E800146E38EC47F04DEF18F003EC4DF00001B3
:1007F800956F03EC4DF00001966F03EC4DF000018E
:10080800986F03EC4DF00001976F03EC4DF0000179
:10081800996F300E136E020E146E38EC47F04DEFE0
:1008280018F003EC4DF00001956F03EC4DF000015A
:10083800966F03EC4DF00001986F03EC4DF000014A
:10084800976F03EC4DF00001996F000E136E020EC6
:10085800146E38EC47F04DEF18F003EC4DF0000142
:10086800996F03EC4DF00001946F03EC4DF003EC2D
:100878004DF003EC4DF00001956F03EC4DF00001D5
:10088800966F03EC4DF00001986F03EC4DF00001FA
:10089800976F03EC4DF0000E136E010E146E38ECDA
:1008A80047F04DEF18F04DEF18F003EC4DF0000154
:1008B800896F500E876F140E856FAEC08BF04DEFA9
:1008C80018F003EC4DF00001896F03EC4DF003ECD8
:1008D8004DF003EC4DF000018951080F876F8951E5
:1008E800F80F856FB0C08BF0BF0E136E000E146E3C
:1008F80016EC4AF04DEF18F0000E0401936F070E46
:10090800936589EF04F08BEF04F08FEF04F04DEF5F
:1009180018F04DEF18F0E50E146EEF0E156E0BEC97
:100928004FF004019351310FA7EC4BF02C0E146ECD
:10093800EF0E156E0BEC4FF0320EA7EC4BF00401E6
:100948009351060D020EF326000EF422C00EF32476
:10095800D96E010EF420DA6EDF500301F46FF45102
:10096800136E146A000E166E0A0E156E7BEC45F0B7
:100978001350310FA7EC4BF0FF0EA7EC4BF0FF0E16
:10098800A7EC4BF0FF0EA7EC4BF0EE0E146EEF0E3B
:10099800156E0BEC4FF004019351310FA7EC4BF09F
:1009A8002C0E146EEF0E156E0BEC4FF0320EA7ECFA
:1009B8004BF004019351060D020EF326000EF422AB
:1009C800C00EF324D96E010EF420DA6EDF50030155
:1009D800F46FF451136E146A000E166E0A0E156E3B
:1009E80061EC46F01350310FA7EC4BF0FF0EA7EC6B
:1009F8004BF0FF0EA7EC4BF0FF0EA7EC4BF0E80E08
:100A0800146EEF0E156E0BEC4FF004019351310F7D
:100A1800A7EC4BF02C0E146EEF0E156E0BEC4FF08E
:100A2800320EA7EC4BF004019351060D040EF32689
:100A3800000EF422C00EF324D96E010EF420DA6EF3
:100A4800DF500301F46FF451136E146A000E166E32
:100A58000A0E156E7BEC45F01350310FA7EC4BF0E6
:100A6800FF0EA7EC4BF0FF0EA7EC4BF0FF0EA7EC28
:100A78004BF0F10E146EEF0E156E0BEC4FF00401F7
:100A88009351310FA7EC4BF02C0E146EEF0E156E30
:100A98000BEC4FF0320EA7EC4BF004019351060D0E
:100AA800040EF326000EF422C00EF324D96E010EB4
:100AB800F420DA6EDF500301F46FF451136E146AF8
:100AC800000E166E0A0E156E61EC46F01350310FCB
:100AD800A7EC4BF0FF0EA7EC4BF0FF0EA7EC4BF08A
:100AE800FF0EA7EC4BF0FA0E146EEF0E156E0BEC22
:100AF8004FF004019351310FA7EC4BF02C0E146EFC
:100B0800EF0E156E0BEC4FF004019351060DC00E5D
:100B1800F324D96E010EF420DA6E450EDE18D8A43F
:100B280098EF05F09AEF05F0A2EF05F0D90E146ED4
:100B3800EF0E156E0BEC4FF0AAEF05F0DC0E146EFD
:100B4800EF0E156E0BEC4FF0AAEF05F0FF0EA7ECB9
:100B58004BF0FF0EA7EC4BF0FF0EA7EC4BF0FC0E92
:100B6800146EEF0E156E0BEC4FF004019351310F1C
:100B7800A7EC4BF02C0E146EEF0E156E0BEC4FF02D
:100B880004019351060D010EF326000EF422C00E47
:100B9800F324D96E010EF420DA6E590EDE18D8A4AB
:100BA800D8EF05F0DAEF05F0E2EF05F0E20E146E8B
:100BB800EF0E156E0BEC4FF0EAEF05F0DF0E146E3A
:100BC800EF0E156E0BEC4FF0EAEF05F0FF0EA7ECF9
:100BD8004BF0FF0EA7EC4BF0FF0EA7EC4BF0040117
:100BE8009351060D050EF326000EF422C00EF324D1
:100BF800D96E010EF420DA6E630EDF6406EF06F09C
:100C080008EF06F06AEF06F0EB0E146EEF0E156EA5
:100C18000BEC4FF004019351310FA7EC4BF02C0E65
:100C2800146EEF0E156E0BEC4FF0D60E146EEF0E21
:100C3800156E0BEC4FF0FF0EA7EC4BF0FF0EA7EC78
:100C48004BF0FF0EA7EC4BF0F40E146EEF0E156E82
:100C58000BEC4FF004019351310FA7EC4BF02C0E25
:100C6800146EEF0E156E0BEC4FF0D30E146EEF0EE4
:100C7800156E0BEC4FF0FF0EA7EC4BF0FF0EA7EC38
:100C88004BF0FF0EA7EC4BF0F70E146EEF0E156E3F
:100C98000BEC4FF004019351310FA7EC4BF02C0EE5
:100CA800146EEF0E156E0BEC4FF0D30E146EEF0EA4
:100CB800156E0BEC4FF0FF0EA7EC4BF0FF0EA7ECF8
:100CC8004BF0FF0EA7EC4BF000EF07F0EB0E146EA5
:100CD800EF0E156E0BEC4FF004019351310FA7EC9A
:100CE8004BF02C0E146EEF0E156E0BEC4FF0D30E6E
:100CF800146EEF0E156E0BEC4FF0FF0EA7EC4BF0D9
:100D0800FF0EA7EC4BF0FF0EA7EC4BF0F40E146EA1
:100D1800EF0E156E0BEC4FF004019351310FA7EC59
:100D28004BF02C0E146EEF0E156E0BEC4FF0320ECE
:100D3800A7EC4BF004019351060D050EF326000EA7
:100D4800F422C00EF324D96E010EF420DA6EDF50BF
:100D58000301F46FF451136E146A000E166E0A0E36
:100D6800156E7BEC45F01350310FA7EC4BF0FF0EDE
:100D7800A7EC4BF0FF0EA7EC4BF0FF0EA7EC4BF0E7
:100D8800F70E146EEF0E156E0BEC4FF00401935135
:100D9800310FA7EC4BF02C0E146EEF0E156E0BEC0A
:100DA8004FF0320EA7EC4BF004019351060D050EDF
:100DB800F326000EF422C00EF324D96E010EF4209F
:100DC800DA6EDF500301F46FF451136E146A000EEB
:100DD800166E0A0E156E61EC46F01350310FA7EC33
:100DE8004BF0FF0EA7EC4BF0FF0EA7EC4BF0FF0EFD
:100DF800A7EC4BF000EF07F00401932B070E936567
:100E080008EF07F00AEF07F08FEF04F04DEF18F046
:100E18004DEF18F0000E936F070E936516EF07F06D
:100E280018EF07F01CEF07F04DEF18F04DEF18F032
:100E3800E50E146EEF0E156E0BEC4FF00401935196
:100E4800310FA7EC4BF02C0E146EEF0E156E0BEC59
:100E58004FF0320EA7EC4BF004019351060D020E31
:100E6800F326000EF422900EF324D96E010EF4201E
:100E7800DA6EDF500301F46FF451136E146A000E3A
:100E8800166E0A0E156E7BEC45F01350310FA7EC69
:100E98004BF0FF0EA7EC4BF0FF0EA7EC4BF0FF0E4C
:100EA800A7EC4BF0EE0E146EEF0E156E0BEC4FF038
:100EB80004019351310FA7EC4BF02C0E146EEF0E7A
:100EC800156E0BEC4FF0320EA7EC4BF0040193516A
:100ED800060D020EF326000EF422900EF324D96EAE
:100EE800010EF420DA6EDF500301F46FF451136E33
:100EF800146A000E166E0A0E156E61EC46F0135059
:100F0800310FA7EC4BF0FF0EA7EC4BF0FF0EA7EC50
:100F18004BF0FF0EA7EC4BF0E80E146EEF0E156EBB
:100F28000BEC4FF004019351310FA7EC4BF02C0E52
:100F3800146EEF0E156E0BEC4FF0320EA7EC4BF063
:100F480004019351060D040EF326000EF422900EB0
:100F5800F324D96E010EF420DA6EDF500301F46F2A
:100F6800F451136E146A000E166E0A0E156E7BECA1
:100F780045F01350310FA7EC4BF0FF0EA7EC4BF0E8
:100F8800FF0EA7EC4BF0FF0EA7EC4BF0F10E146E22
:100F9800EF0E156E0BEC4FF004019351310FA7ECD7
:100FA8004BF02C0E146EEF0E156E0BEC4FF0320E4C
:100FB800A7EC4BF004019351060D040EF326000E26
:100FC800F422900EF324D96E010EF420DA6EDF506D
:100FD8000301F46FF451136E146A000E166E0A0EB4
:100FE800156E61EC46F01350310FA7EC4BF0FF0E75
:100FF800A7EC4BF0FF0EA7EC4BF0FF0EA7EC4BF065
:10100800FA0E146EEF0E156E0BEC4FF004019351AF
:10101800310FA7EC4BF02C0E146EEF0E156E0BEC87
:101028004FF004019351060D900EF324D96E010E72
:10103800F420DA6E450EDE18D8A425EF08F027EF65
:1010480008F02FEF08F0D90E146EEF0E156E0BECAA
:101058004FF037EF08F0DC0E146EEF0E156E0BEC48
:101068004FF037EF08F0FF0EA7EC4BF0FF0EA7ECA0
:101078004BF0FF0EA7EC4BF0FC0E146EEF0E156E46
:101088000BEC4FF004019351310FA7EC4BF02C0EF1
:10109800146EEF0E156E0BEC4FF004019351060D14
:1010A800010EF326000EF422900EF324D96E010EE1
:1010B800F420DA6E590EDE18D8A465EF08F067EF51
:1010C80008F06FEF08F0E20E146EEF0E156E0BECE1
:1010D8004FF077EF08F0DF0E146EEF0E156E0BEC85
:1010E8004FF077EF08F0FF0EA7EC4BF0FF0EA7ECE0
:1010F8004BF0FF0EA7EC4BF004019351060D050EC3
:10110800F326000EF422900EF324D96E010EF4207B
:10111800DA6E630EDF6493EF08F095EF08F0F7EFEF
:1011280008F0EB0E146EEF0E156E0BEC4FF0040189
:101138009351310FA7EC4BF02C0E146EEF0E156E79
:101148000BEC4FF0D60E146EEF0E156E0BEC4FF045
:10115800FF0EA7EC4BF0FF0EA7EC4BF0FF0EA7EC31
:101168004BF0F40E146EEF0E156E0BEC4FF00401FD
:101178009351310FA7EC4BF02C0E146EEF0E156E39
:101188000BEC4FF0D30E146EEF0E156E0BEC4FF008
:10119800FF0EA7EC4BF0FF0EA7EC4BF0FF0EA7ECF1
:1011A8004BF0F70E146EEF0E156E0BEC4FF00401BA
:1011B8009351310FA7EC4BF02C0E146EEF0E156EF9
:1011C8000BEC4FF0D30E146EEF0E156E0BEC4FF0C8
:1011D800FF0EA7EC4BF0FF0EA7EC4BF0FF0EA7ECB1
:1011E8004BF08DEF09F0EB0E146EEF0E156E0BEC55
:1011F8004FF004019351310FA7EC4BF02C0E146EF5
:10120800EF0E156E0BEC4FF0D30E146EEF0E156E3D
:101218000BEC4FF0FF0EA7EC4BF0FF0EA7EC4BF0DA
:10122800FF0EA7EC4BF0F40E146EEF0E156E0BECE0
:101238004FF004019351310FA7EC4BF02C0E146EB4
:10124800EF0E156E0BEC4FF0320EA7EC4BF00401CD
:101258009351060D050EF326000EF422900EF3248A
:10126800D96E010EF420DA6EDF500301F46FF451E9
:10127800136E146A000E166E0A0E156E7BEC45F09E
:101288001350310FA7EC4BF0FF0EA7EC4BF0FF0EFD
:10129800A7EC4BF0FF0EA7EC4BF0F70E146EEF0E19
:1012A800156E0BEC4FF004019351310FA7EC4BF086
:1012B8002C0E146EEF0E156E0BEC4FF0320EA7ECE1
:1012C8004BF004019351060D050EF326000EF4228F
:1012D800900EF324D96E010EF420DA6EDF5003016C
:1012E800F46FF451136E146A000E166E0A0E156E22
:1012F80061EC46F01350310FA7EC4BF0FF0EA7EC52
:101308004BF0FF0EA7EC4BF0FF0EA7EC4BF08DEF68
:1013180009F00401932B070E936595EF09F097EFF9
:1013280009F01CEF07F04DEF18F04DEF18F0000E24
:10133800936F070E9365A3EF09F0A5EF09F0A9EFE6
:1013480009F04DEF18F04DEF18F0E50E146EEF0EA2
:10135800156E0BEC4FF004019351310FA7EC4BF0D5
:101368002C0E146EEF0E156E0BEC4FF0320EA7EC30
:101378004BF004019351060D020EF326000EF422E1
:10138800600EF324D96E010EF420DA6EDF500301EB
:10139800F46FF451136E146A000E166E0A0E156E71
:1013A8007BEC45F01350310FA7EC4BF0FF0EA7EC88
:1013B8004BF0FF0EA7EC4BF0FF0EA7EC4BF0EE0E38
:1013C800146EEF0E156E0BEC4FF004019351310FB4
:1013D800A7EC4BF02C0E146EEF0E156E0BEC4FF0C5
:1013E800320EA7EC4BF004019351060D020EF326C2
:1013F800000EF422600EF324D96E010EF420DA6E8A
:10140800DF500301F46FF451136E146A000E166E68
:101418000A0E156E61EC46F01350310FA7EC4BF035
:10142800FF0EA7EC4BF0FF0EA7EC4BF0FF0EA7EC5E
:101438004BF0E80E146EEF0E156E0BEC4FF0040136
:101448009351310FA7EC4BF02C0E146EEF0E156E66
:101458000BEC4FF0320EA7EC4BF004019351060D44
:10146800040EF326000EF422600EF324D96E010E4A
:10147800F420DA6EDF500301F46FF451136E146A2E
:10148800000E166E0A0E156E7BEC45F01350310FE8
:10149800A7EC4BF0FF0EA7EC4BF0FF0EA7EC4BF0C0
:1014A800FF0EA7EC4BF0F10E146EEF0E156E0BEC61
:1014B8004FF004019351310FA7EC4BF02C0E146E32
:1014C800EF0E156E0BEC4FF0320EA7EC4BF004014B
:1014D8009351060D040EF326000EF422600EF32439
:1014E800D96E010EF420DA6EDF500301F46FF45167
:1014F800136E146A000E166E0A0E156E61EC46F035
:101508001350310FA7EC4BF0FF0EA7EC4BF0FF0E7A
:10151800A7EC4BF0FF0EA7EC4BF0FA0E146EEF0E93
:10152800156E0BEC4FF004019351310FA7EC4BF003
:101538002C0E146EEF0E156E0BEC4FF00401935148
:10154800060D600EF324D96E010EF420DA6E450EF6
:10155800DE18D8A4B2EF0AF0B4EF0AF0BCEF0AF034
:10156800D90E146EEF0E156E0BEC4FF0C4EF0AF0A7
:10157800DC0E146EEF0E156E0BEC4FF0C4EF0AF094
:10158800FF0EA7EC4BF0FF0EA7EC4BF0FF0EA7ECFD
:101598004BF0FC0E146EEF0E156E0BEC4FF00401C1
:1015A8009351310FA7EC4BF02C0E146EEF0E156E05
:1015B8000BEC4FF004019351060D010EF326000EBB
:1015C800F422600EF324D96E010EF420DA6E590E5F
:1015D800DE18D8A4F2EF0AF0F4EF0AF0FCEF0AF0F4
:1015E800E20E146EEF0E156E0BEC4FF004EF0BF0DD
:1015F800DF0E146EEF0E156E0BEC4FF004EF0BF0D0
:10160800FF0EA7EC4BF0FF0EA7EC4BF0FF0EA7EC7C
:101618004BF004019351060D050EF326000EF4223B
:10162800600EF324D96E010EF420DA6E630EDF64C7
:1016380020EF0BF022EF0BF084EF0BF0EB0E146EA3
:10164800EF0E156E0BEC4FF004019351310FA7EC20
:101658004BF02C0E146EEF0E156E0BEC4FF0D60EF1
:10166800146EEF0E156E0BEC4FF0FF0EA7EC4BF05F
:10167800FF0EA7EC4BF0FF0EA7EC4BF0F40E146E28
:10168800EF0E156E0BEC4FF004019351310FA7ECE0
:101698004BF02C0E146EEF0E156E0BEC4FF0D30EB4
:1016A800146EEF0E156E0BEC4FF0FF0EA7EC4BF01F
:1016B800FF0EA7EC4BF0FF0EA7EC4BF0F70E146EE5
:1016C800EF0E156E0BEC4FF004019351310FA7ECA0
:1016D8004BF02C0E146EEF0E156E0BEC4FF0D30E74
:1016E800146EEF0E156E0BEC4FF0FF0EA7EC4BF0DF
:1016F800FF0EA7EC4BF0FF0EA7EC4BF01AEF0CF027
:10170800EB0E146EEF0E156E0BEC4FF004019351B7
:10171800310FA7EC4BF02C0E146EEF0E156E0BEC80
:101728004FF0D30E146EEF0E156E0BEC4FF0FF0E4C
:10173800A7EC4BF0FF0EA7EC4BF0FF0EA7EC4BF01D
:10174800F40E146EEF0E156E0BEC4FF0040193516E
:10175800310FA7EC4BF02C0E146EEF0E156E0BEC40
:101768004FF0320EA7EC4BF004019351060D050E15
:10177800F326000EF422600EF324D96E010EF42035
:10178800DA6EDF500301F46FF451136E146A000E21
:10179800166E0A0E156E7BEC45F01350310FA7EC50
:1017A8004BF0FF0EA7EC4BF0FF0EA7EC4BF0FF0E33
:1017B800A7EC4BF0F70E146EEF0E156E0BEC4FF016
:1017C80004019351310FA7EC4BF02C0E146EEF0E61
:1017D800156E0BEC4FF0320EA7EC4BF00401935151
:1017E800060D050EF326000EF422600EF324D96EC2
:1017F800010EF420DA6EDF500301F46FF451136E1A
:10180800146A000E166E0A0E156E61EC46F013503F
:10181800310FA7EC4BF0FF0EA7EC4BF0FF0EA7EC37
:101828004BF0FF0EA7EC4BF01AEF0CF00401932BD2
:10183800070E936522EF0CF024EF0CF0A9EF09F0E6
:101848004DEF18F04DEF18F0000E936F070E9365EB
:1018580030EF0CF032EF0CF036EF0CF04DEF18F0E3
:101868004DEF18F0E50E146EEF0E156E0BEC4FF001
:1018780004019351310FA7EC4BF02C0E146EEF0EB0
:10188800156E0BEC4FF0320EA7EC4BF004019351A0
:10189800060D020EF326000EF422900EF324D96EE4
:1018A800020EF420DA6EDF500301F46FF451136E68
:1018B800146A000E166E0A0E156E7BEC45F0135076
:1018C800310FA7EC4BF0FF0EA7EC4BF0FF0EA7EC87
:1018D8004BF0FF0EA7EC4BF0EE0E146EEF0E156EEC
:1018E8000BEC4FF004019351310FA7EC4BF02C0E89
:1018F800146EEF0E156E0BEC4FF0320EA7EC4BF09A
:1019080004019351060D020EF326000EF422900EE8
:10191800F324D96E020EF420DA6EDF500301F46F5F
:10192800F451136E146A000E166E0A0E156E61ECF1
:1019380046F01350310FA7EC4BF0FF0EA7EC4BF01D
:10194800FF0EA7EC4BF0FF0EA7EC4BF0E80E146E61
:10195800EF0E156E0BEC4FF004019351310FA7EC0D
:101968004BF02C0E146EEF0E156E0BEC4FF0320E82
:10197800A7EC4BF004019351060D040EF326000E5C
:10198800F422900EF324D96E020EF420DA6EDF50A2
:101998000301F46FF451136E146A000E166E0A0EEA
:1019A800156E7BEC45F01350310FA7EC4BF0FF0E92
:1019B800A7EC4BF0FF0EA7EC4BF0FF0EA7EC4BF09B
:1019C800F10E146EEF0E156E0BEC4FF004019351EF
:1019D800310FA7EC4BF02C0E146EEF0E156E0BECBE
:1019E8004FF0320EA7EC4BF004019351060D040E94
:1019F800F326000EF422900EF324D96E020EF42082
:101A0800DA6EDF500301F46FF451136E146A000E9E
:101A1800166E0A0E156E61EC46F01350310FA7ECE6
:101A28004BF0FF0EA7EC4BF0FF0EA7EC4BF0FF0EB0
:101A3800A7EC4BF0FC0E146EEF0E156E0BEC4FF08E
:101A480004019351310FA7EC4BF02C0E146EEF0EDE
:101A5800156E0BEC4FF004019351060D010EF326A1
:101A6800000EF422900EF324D96E020EF420DA6EE2
:101A7800590EDE18D8A443EF0DF045EF0DF04DEFE9
:101A88000DF0E20E146EEF0E156E0BEC4FF055EFE5
:101A98000DF0DF0E146EEF0E156E0BEC4FF055EFD8
:101AA8000DF0FF0EA7EC4BF0FF0EA7EC4BF0FF0E6E
:101AB800A7EC4BF00401932B070E936566EF0DF02E
:101AC80068EF0DF036EF0CF04DEF18F04DEF18F011
:101AD800000E936F070E936574EF0DF076EF0DF01F
:101AE8007AEF0DF04DEF18F04DEF18F0E50E146E8B
:101AF800EF0E156E0BEC4FF004019351310FA7EC6C
:101B08004BF02C0E146EEF0E156E0BEC4FF0320EE0
:101B1800A7EC4BF004019351060D020EF326000EBC
:101B2800F422600EF324D96E020EF420DA6EDF5030
:101B38000301F46FF451136E146A000E166E0A0E48
:101B4800156E7BEC45F01350310FA7EC4BF0FF0EF0
:101B5800A7EC4BF0FF0EA7EC4BF0FF0EA7EC4BF0F9
:101B6800EE0E146EEF0E156E0BEC4FF00401935150
:101B7800310FA7EC4BF02C0E146EEF0E156E0BEC1C
:101B88004FF0320EA7EC4BF004019351060D020EF4
:101B9800F326000EF422600EF324D96E020EF42010
:101BA800DA6EDF500301F46FF451136E146A000EFD
:101BB800166E0A0E156E61EC46F01350310FA7EC45
:101BC8004BF0FF0EA7EC4BF0FF0EA7EC4BF0FF0E0F
:101BD800A7EC4BF0E80E146EEF0E156E0BEC4FF001
:101BE80004019351310FA7EC4BF02C0E146EEF0E3D
:101BF800156E0BEC4FF0320EA7EC4BF0040193512D
:101C0800060D040EF326000EF422600EF324D96E9E
:101C1800020EF420DA6EDF500301F46FF451136EF4
:101C2800146A000E166E0A0E156E7BEC45F0135002
:101C3800310FA7EC4BF0FF0EA7EC4BF0FF0EA7EC13
:101C48004BF0FF0EA7EC4BF0F10E146EEF0E156E75
:101C58000BEC4FF004019351310FA7EC4BF02C0E15
:101C6800146EEF0E156E0BEC4FF0320EA7EC4BF026
:101C780004019351060D040EF326000EF422600EA3
:101C8800F324D96E020EF420DA6EDF500301F46FEC
:101C9800F451136E146A000E166E0A0E156E61EC7E
:101CA80046F01350310FA7EC4BF0FF0EA7EC4BF0AA
:101CB800FF0EA7EC4BF0FF0EA7EC4BF0FC0E146EDA
:101CC800EF0E156E0BEC4FF004019351310FA7EC9A
:101CD8004BF02C0E146EEF0E156E0BEC4FF004014A
:101CE8009351060D010EF326000EF422600EF32424
:101CF800D96E020EF420DA6E590EDE18D8A487EFDA
:101D08000EF089EF0EF091EF0EF0E20E146EEF0E6A
:101D1800156E0BEC4FF099EF0EF0DF0E146EEF0E10
:101D2800156E0BEC4FF099EF0EF0FF0EA7EC4BF091
:101D3800FF0EA7EC4BF0FF0EA7EC4BF00401932B22
:101D4800070E9365AAEF0EF0ACEF0EF07AEF0DF0E8
:101D58004DEF18F04DEF18F0000E936F070E9365D6
:101D6800B8EF0EF0BAEF0EF0BEEF0EF04DEF18F030
:101D78004DEF18F0E50E146EEF0E156E0BEC4FF0EC
:101D880004019351310FA7EC4BF02C0E146EEF0E9B
:101D9800156E0BEC4FF0320EA7EC4BF0040193518B
:101DA800060D020EF326000EF422300EF324D96E2F
:101DB800010EF420DA6EDF500301F46FF451136E54
:101DC800146A000E166E0A0E156E7BEC45F0135061
:101DD800310FA7EC4BF0FF0EA7EC4BF0FF0EA7EC72
:101DE8004BF0FF0EA7EC4BF0EE0E146EEF0E156ED7
:101DF8000BEC4FF004019351310FA7EC4BF02C0E74
:101E0800146EEF0E156E0BEC4FF0320EA7EC4BF084
:101E180004019351060D020EF326000EF422300E33
:101E2800F324D96E010EF420DA6EDF500301F46F4B
:101E3800F451136E146A000E166E0A0E156E61ECDC
:101E480046F01350310FA7EC4BF0FF0EA7EC4BF008
:101E5800FF0EA7EC4BF0FF0EA7EC4BF0E80E146E4C
:101E6800EF0E156E0BEC4FF004019351310FA7ECF8
:101E78004BF02C0E146EEF0E156E0BEC4FF0320E6D
:101E8800A7EC4BF004019351060D040EF326000E47
:101E9800F422300EF324D96E010EF420DA6EDF50EE
:101EA8000301F46FF451136E146A000E166E0A0ED5
:101EB800156E7BEC45F01350310FA7EC4BF0FF0E7D
:101EC800A7EC4BF0FF0EA7EC4BF0FF0EA7EC4BF086
:101ED800F10E146EEF0E156E0BEC4FF004019351DA
:101EE800310FA7EC4BF02C0E146EEF0E156E0BECA9
:101EF8004FF0320EA7EC4BF004019351060D040E7F
:101F0800F326000EF422300EF324D96E010EF420CD
:101F1800DA6EDF500301F46FF451136E146A000E89
:101F2800166E0A0E156E61EC46F01350310FA7ECD1
:101F38004BF0FF0EA7EC4BF0FF0EA7EC4BF0FF0E9B
:101F4800A7EC4BF0FC0E146EEF0E156E0BEC4FF079
:101F580004019351310FA7EC4BF02C0E146EEF0EC9
:101F6800156E0BEC4FF004019351060D010EF3268C
:101F7800000EF422300EF324D96E010EF420DA6E2E
:101F8800590EDE18D8A4CBEF0FF0CDEF0FF0D5EF38
:101F98000FF0E20E146EEF0E156E0BEC4FF0DDEF46
:101FA8000FF0DF0E146EEF0E156E0BEC4FF0DDEF39
:101FB8000FF0FF0EA7EC4BF0FF0EA7EC4BF0FF0E57
:101FC800A7EC4BF004019351060D050EF326000E05
:101FD800F422300EF324D96E010EF420DA6E630E6B
:101FE800DF64F9EF0FF0FBEF0FF05DEF10F0EB0E91
:101FF800146EEF0E156E0BEC4FF004019351310F78
:10200800A7EC4BF02C0E146EEF0E156E0BEC4FF088
:10201800D60E146EEF0E156E0BEC4FF0FF0EA7ECFC
:102028004BF0FF0EA7EC4BF0FF0EA7EC4BF0F40EB5
:10203800146EEF0E156E0BEC4FF004019351310F37
:10204800A7EC4BF02C0E146EEF0E156E0BEC4FF048
:10205800D30E146EEF0E156E0BEC4FF0FF0EA7ECBF
:102068004BF0FF0EA7EC4BF0FF0EA7EC4BF0F70E72
:10207800146EEF0E156E0BEC4FF004019351310FF7
:10208800A7EC4BF02C0E146EEF0E156E0BEC4FF008
:10209800D30E146EEF0E156E0BEC4FF0FF0EA7EC7F
:1020A8004BF0FF0EA7EC4BF0FF0EA7EC4BF0F3EF55
:1020B80010F0EB0E146EEF0E156E0BEC4FF00401E2
:1020C8009351310FA7EC4BF02C0E146EEF0E156EDA
:1020D8000BEC4FF0D30E146EEF0E156E0BEC4FF0A9
:1020E800FF0EA7EC4BF0FF0EA7EC4BF0FF0EA7EC92
:1020F8004BF0F40E146EEF0E156E0BEC4FF004015E
:102108009351310FA7EC4BF02C0E146EEF0E156E99
:102118000BEC4FF0320EA7EC4BF004019351060D77
:10212800050EF326000EF422300EF324D96E010EAC
:10213800F420DA6EDF500301F46FF451136E146A61
:10214800000E166E0A0E156E7BEC45F01350310F1B
:10215800A7EC4BF0FF0EA7EC4BF0FF0EA7EC4BF0F3
:10216800FF0EA7EC4BF0F70E146EEF0E156E0BEC8E
:102178004FF004019351310FA7EC4BF02C0E146E65
:10218800EF0E156E0BEC4FF0320EA7EC4BF004017E
:102198009351060D050EF326000EF422300EF3249B
:1021A800D96E010EF420DA6EDF500301F46FF4519A
:1021B800136E146A000E166E0A0E156E61EC46F068
:1021C8001350310FA7EC4BF0FF0EA7EC4BF0FF0EAE
:1021D800A7EC4BF0FF0EA7EC4BF0F3EF10F0040167
:1021E800932B070E9365FBEF10F0FDEF10F0BEEF99
:1021F8000EF04DEF18F04DEF18F0000E936F070E2C
:10220800936509EF11F00BEF11F00FEF11F04DEF9F
:1022180018F04DEF18F0E50E146EEF0E156E0BEC7E
:102228004FF004019351310FA7EC4BF02C0E146EB4
:10223800EF0E156E0BEC4FF0320EA7EC4BF00401CD
:102248009351060D020EF326000EF422300EF324ED
:10225800D96E020EF420DA6EDF500301F46FF451E8
:10226800136E146A000E166E0A0E156E7BEC45F09E
:102278001350310FA7EC4BF0FF0EA7EC4BF0FF0EFD
:10228800A7EC4BF0FF0EA7EC4BF0EE0E146EEF0E22
:10229800156E0BEC4FF004019351310FA7EC4BF086
:1022A8002C0E146EEF0E156E0BEC4FF0320EA7ECE1
:1022B8004BF004019351060D020EF326000EF42292
:1022C800300EF324D96E020EF420DA6EDF500301CB
:1022D800F46FF451136E146A000E166E0A0E156E22
:1022E80061EC46F01350310FA7EC4BF0FF0EA7EC52
:1022F8004BF0FF0EA7EC4BF0FF0EA7EC4BF0E80EEF
:10230800146EEF0E156E0BEC4FF004019351310F64
:10231800A7EC4BF02C0E146EEF0E156E0BEC4FF075
:10232800320EA7EC4BF004019351060D040EF32670
:10233800000EF422300EF324D96E020EF420DA6E69
:10234800DF500301F46FF451136E146A000E166E19
:102358000A0E156E7BEC45F01350310FA7EC4BF0CD
:10236800FF0EA7EC4BF0FF0EA7EC4BF0FF0EA7EC0F
:102378004BF0F10E146EEF0E156E0BEC4FF00401DE
:102388009351310FA7EC4BF02C0E146EEF0E156E17
:102398000BEC4FF0320EA7EC4BF004019351060DF5
:1023A800040EF326000EF422300EF324D96E020E2A
:1023B800F420DA6EDF500301F46FF451136E146ADF
:1023C800000E166E0A0E156E61EC46F01350310FB2
:1023D800A7EC4BF0FF0EA7EC4BF0FF0EA7EC4BF071
:1023E800FF0EA7EC4BF0FC0E146EEF0E156E0BEC07
:1023F8004FF004019351310FA7EC4BF02C0E146EE3
:10240800EF0E156E0BEC4FF004019351060D010E03
:10241800F326000EF422300EF324D96E020EF420B7
:10242800DA6E590EDE18D8A41CEF12F01EEF12F067
:1024380026EF12F0E20E146EEF0E156E0BEC4FF055
:102448002EEF12F0DF0E146EEF0E156E0BEC4FF040
:102458002EEF12F0FF0EA7EC4BF0FF0EA7EC4BF09F
:10246800FF0EA7EC4BF004019351060D050EF32661
:10247800000EF422300EF324D96E020EF420DA6E28
:10248800630EDF644AEF12F04CEF12F0AEEF12F079
:10249800EB0E146EEF0E156E0BEC4FF0040193511A
:1024A800310FA7EC4BF02C0E146EEF0E156E0BECE3
:1024B8004FF0D60E146EEF0E156E0BEC4FF0FF0EAC
:1024C800A7EC4BF0FF0EA7EC4BF0FF0EA7EC4BF080
:1024D800F40E146EEF0E156E0BEC4FF004019351D1
:1024E800310FA7EC4BF02C0E146EEF0E156E0BECA3
:1024F8004FF0D30E146EEF0E156E0BEC4FF0FF0E6F
:10250800A7EC4BF0FF0EA7EC4BF0FF0EA7EC4BF03F
:10251800F70E146EEF0E156E0BEC4FF0040193518D
:10252800310FA7EC4BF02C0E146EEF0E156E0BEC62
:102538004FF0D30E146EEF0E156E0BEC4FF0FF0E2E
:10254800A7EC4BF0FF0EA7EC4BF0FF0EA7EC4BF0FF
:1025580044EF13F0EB0E146EEF0E156E0BEC4FF00C
:1025680004019351310FA7EC4BF02C0E146EEF0EB3
:10257800156E0BEC4FF0D30E146EEF0E156E0BECC0
:102588004FF0FF0EA7EC4BF0FF0EA7EC4BF0FF0E41
:10259800A7EC4BF0F40E146EEF0E156E0BEC4FF02B
:1025A80004019351310FA7EC4BF02C0E146EEF0E73
:1025B800156E0BEC4FF0320EA7EC4BF00401935163
:1025C800060D050EF326000EF422300EF324D96E04
:1025D800020EF420DA6EDF500301F46FF451136E2B
:1025E800146A000E166E0A0E156E7BEC45F0135039
:1025F800310FA7EC4BF0FF0EA7EC4BF0FF0EA7EC4A
:102608004BF0FF0EA7EC4BF0F70E146EEF0E156EA5
:102618000BEC4FF004019351310FA7EC4BF02C0E4B
:10262800146EEF0E156E0BEC4FF0320EA7EC4BF05C
:1026380004019351060D050EF326000EF422300E08
:10264800F324D96E020EF420DA6EDF500301F46F22
:10265800F451136E146A000E166E0A0E156E61ECB4
:1026680046F01350310FA7EC4BF0FF0EA7EC4BF0E0
:10267800FF0EA7EC4BF0FF0EA7EC4BF044EF13F066
:102688000401932B070E93654CEF13F04EEF13F0F4
:102698000FEF11F04DEF18F04DEF18F0000E936F9B
:1026A800070E93655AEF13F05CEF13F060EF13F029
:1026B8004DEF18F04DEF18F0E50E146EEF0E156E95
:1026C8000BEC4FF004019351310FA7EC4BF02C0E9B
:1026D800146EEF0E156E0BEC4FF0320EA7EC4BF0AC
:1026E80004019351060D020EF326000EF422000E8B
:1026F800F324D96E020EF420DA6EDF500301F46F72
:10270800F451136E146A000E166E0A0E156E7BECE9
:1027180045F01350310FA7EC4BF0FF0EA7EC4BF030
:10272800FF0EA7EC4BF0FF0EA7EC4BF0EE0E146E6D
:10273800EF0E156E0BEC4FF004019351310FA7EC1F
:102748004BF02C0E146EEF0E156E0BEC4FF0320E94
:10275800A7EC4BF004019351060D020EF326000E70
:10276800F422000EF324D96E020EF420DA6EDF5044
:102778000301F46FF451136E146A000E166E0A0EFC
:10278800156E61EC46F01350310FA7EC4BF0FF0EBD
:10279800A7EC4BF0FF0EA7EC4BF0FF0EA7EC4BF0AD
:1027A800E80E146EEF0E156E0BEC4FF0040193510A
:1027B800310FA7EC4BF02C0E146EEF0E156E0BECD0
:1027C8004FF0320EA7EC4BF004019351060D040EA6
:1027D800F326000EF422000EF324D96E020EF42024
:1027E800DA6EDF500301F46FF451136E146A000EB1
:1027F800166E0A0E156E7BEC45F01350310FA7ECE0
:102808004BF0FF0EA7EC4BF0FF0EA7EC4BF0FF0EC2
:10281800A7EC4BF0F10E146EEF0E156E0BEC4FF0AB
:1028280004019351310FA7EC4BF02C0E146EEF0EF0
:10283800156E0BEC4FF0320EA7EC4BF004019351E0
:10284800060D040EF326000EF422000EF324D96EB2
:10285800020EF420DA6EDF500301F46FF451136EA8
:10286800146A000E166E0A0E156E61EC46F01350CF
:10287800310FA7EC4BF0FF0EA7EC4BF0FF0EA7ECC7
:102888004BF0FF0EA7EC4BF0FC0E146EEF0E156E1E
:102898000BEC4FF004019351310FA7EC4BF02C0EC9
:1028A800146EEF0E156E0BEC4FF004019351060DEC
:1028B800010EF326000EF422000EF324D96E020E48
:1028C800F420DA6E590EDE18D8A46DEF14F06FEF0D
:1028D80014F077EF14F0E20E146EEF0E156E0BEC99
:1028E8004FF07FEF14F0DF0E146EEF0E156E0BEC49
:1028F8004FF07FEF14F0FF0EA7EC4BF0FF0EA7ECA4
:102908004BF0FF0EA7EC4BF004019351060D050E9A
:10291800F326000EF422000EF324D96E020EF420E2
:10292800DA6E630EDF649BEF14F09DEF14F0FFEF97
:1029380014F0EB0E146EEF0E156E0BEC4FF0040155
:102948009351310FA7EC4BF02C0E146EEF0E156E51
:102958000BEC4FF0D60E146EEF0E156E0BEC4FF01D
:10296800FF0EA7EC4BF0FF0EA7EC4BF0FF0EA7EC09
:102978004BF0F40E146EEF0E156E0BEC4FF00401D5
:102988009351310FA7EC4BF02C0E146EEF0E156E11
:102998000BEC4FF0D30E146EEF0E156E0BEC4FF0E0
:1029A800FF0EA7EC4BF0FF0EA7EC4BF0FF0EA7ECC9
:1029B8004BF0F70E146EEF0E156E0BEC4FF0040192
:1029C8009351310FA7EC4BF02C0E146EEF0E156ED1
:1029D8000BEC4FF0D30E146EEF0E156E0BEC4FF0A0
:1029E800FF0EA7EC4BF0FF0EA7EC4BF0FF0EA7EC89
:1029F8004BF095EF15F0EB0E146EEF0E156E0BEC19
:102A08004FF004019351310FA7EC4BF02C0E146ECC
:102A1800EF0E156E0BEC4FF0D30E146EEF0E156E15
:102A28000BEC4FF0FF0EA7EC4BF0FF0EA7EC4BF0B2
:102A3800FF0EA7EC4BF0F40E146EEF0E156E0BECB8
:102A48004FF004019351310FA7EC4BF02C0E146E8C
:102A5800EF0E156E0BEC4FF0320EA7EC4BF00401A5
:102A68009351060D050EF326000EF422000EF324F2
:102A7800D96E020EF420DA6EDF500301F46FF451C0
:102A8800136E146A000E166E0A0E156E7BEC45F076
:102A98001350310FA7EC4BF0FF0EA7EC4BF0FF0ED5
:102AA800A7EC4BF0FF0EA7EC4BF0F70E146EEF0EF1
:102AB800156E0BEC4FF004019351310FA7EC4BF05E
:102AC8002C0E146EEF0E156E0BEC4FF0320EA7ECB9
:102AD8004BF004019351060D050EF326000EF42267
:102AE800000EF324D96E020EF420DA6EDF500301D3
:102AF800F46FF451136E146A000E166E0A0E156EFA
:102B080061EC46F01350310FA7EC4BF0FF0EA7EC29
:102B18004BF0FF0EA7EC4BF0FF0EA7EC4BF095EF38
:102B280015F00401932B070E93659DEF15F09FEFA9
:102B380015F060EF13F04DEF18F04DEF18F0000EA0
:102B4800936F070E9365ABEF15F0ADEF15F0B1EF8E
:102B580015F04DEF18F04DEF18F0E50E146EEF0E6E
:102B6800156E0BEC4FF004019351310FA7EC4BF0AD
:102B78002C0E146EEF0E156E0BEC4FF0320EA7EC08
:102B88004BF004019351060D020EF326000EF422B9
:102B9800000EF324D96E010EF420DA6EDF50030123
:102BA800F46FF451136E146A000E166E0A0E156E49
:102BB8007BEC45F01350310FA7EC4BF0FF0EA7EC60
:102BC8004BF0FF0EA7EC4BF0FF0EA7EC4BF0EE0E10
:102BD800146EEF0E156E0BEC4FF004019351310F8C
:102BE800A7EC4BF02C0E146EEF0E156E0BEC4FF09D
:102BF800320EA7EC4BF004019351060D020EF3269A
:102C0800000EF422000EF324D96E010EF420DA6EC1
:102C1800DF500301F46FF451136E146A000E166E40
:102C28000A0E156E61EC46F01350310FA7EC4BF00D
:102C3800FF0EA7EC4BF0FF0EA7EC4BF0FF0EA7EC36
:102C48004BF0E80E146EEF0E156E0BEC4FF004010E
:102C58009351310FA7EC4BF02C0E146EEF0E156E3E
:102C68000BEC4FF0320EA7EC4BF004019351060D1C
:102C7800040EF326000EF422000EF324D96E010E82
:102C8800F420DA6EDF500301F46FF451136E146A06
:102C9800000E166E0A0E156E7BEC45F01350310FC0
:102CA800A7EC4BF0FF0EA7EC4BF0FF0EA7EC4BF098
:102CB800FF0EA7EC4BF0F10E146EEF0E156E0BEC39
:102CC8004FF004019351310FA7EC4BF02C0E146E0A
:102CD800EF0E156E0BEC4FF0320EA7EC4BF0040123
:102CE8009351060D040EF326000EF422000EF32471
:102CF800D96E010EF420DA6EDF500301F46FF4513F
:102D0800136E146A000E166E0A0E156E61EC46F00C
:102D18001350310FA7EC4BF0FF0EA7EC4BF0FF0E52
:102D2800A7EC4BF0FF0EA7EC4BF0F80E146EEF0E6D
:102D3800156E0BEC4FF004019351310FA7EC4BF0DB
:102D4800CD0E146EEF0E156E0BEC4FF0040193517F
:102D5800060D050EF326000EF422000EF324D96E9C
:102D6800010EF420DA6EDF500301F46F0401935171
:102D7800060D000EF324D96E010EF420DA6EDF5032
:102D88000301F56FF45104018B6FF5C38CF4000E49
:102D98008D6F000E8E6F000E8F6F000E906F11EF0B
:102DA80017F08BC413F08CC414F0000E166E0A0EC4
:102DB800156E55EC4AF0135004018A6F8DC413F058
:102DC8008EC414F08FC415F090C416F00A0E176E56
:102DD800000E186E000E196E000E1A6ECBEC4AF03B
:102DE80004018A5113248D6F000E14208E6F000E7B
:102DF80015208F6F000E1620906F8BC413F08CC4B3
:102E080014F0000E166E0A0E156E4FEC49F013C042
:102E18008BF414C08CF411EF17F004018B518C1152
:102E2800D8A419EF17F01BEF17F0D5EF16F054EFF1
:102E380017F054EF17F08DC413F08EC414F08FC43C
:102E480015F090C416F00A0E176E000E186E000EDC
:102E5800196E000E1A6E01EC49F0135004018A6FC6
:102E68008A51300FA7EC4BF08DC413F08EC414F0C8
:102E78008FC415F090C416F00A0E176E000E186E67
:102E8800000E196E000E1A6EA1EC47F013C08DF4F7
:102E980014C08EF415C08FF416C090F454EF17F0D8
:102EA80004018D518E118F119011D8A45EEF17F087
:102EB80060EF17F01FEF17F062EF17F0FF0EA7ECA7
:102EC8004BF0FF0EA7EC4BF0FF0EA7EC4BF0FC0EFF
:102ED800146EEF0E156E0BEC4FF004019351310F89
:102EE800A7EC4BF02C0E146EEF0E156E0BEC4FF09A
:102EF80004019351060D010EF326000EF422000E74
:102F0800F324D96E010EF420DA6E590EDE18D8A417
:102F180090EF17F092EF17F09AEF17F0E20E146E99
:102F2800EF0E156E0BEC4FF0A2EF17F0DF0E146EDC
:102F3800EF0E156E0BEC4FF0A2EF17F0FF0EA7EC9B
:102F48004BF0FF0EA7EC4BF0FF0EA7EC4BF0040183
:102F5800932B070E9365B3EF17F0B5EF17F0B1EFAA
:102F680015F04DEF18F04DEF18F04DEF18F08951AE
:102F7800410AD8B480EF04F0030AD8B40EEF07F082
:102F8800010AD8B49BEF09F0070AD8B428EF0CF06F
:102F9800010AD8B46CEF0DF0030AD8B4B0EF0EF004
:102FA800010AD8B401EF11F00F0AD8B452EF13F0A8
:102FB800010AD8B4A3EF15F0060AD8B434EF03F029
:102FC8001D0AD8B438EF03F0010AD8B441EF03F072
:102FD800090AD8B431EF03F03B0AD8B445EF03F03F
:102FE800030AD8B465EF03F0010AD8B485EF03F0FB
:102FF800070AD8B4A5EF03F0010AD8B4C1EF03F06B
:10300800030AD8B4DDEF03F0010AD8B4F9EF03F0EE
:103018000F0AD8B415EF04F0010AD8B431EF04F060
:10302800190AD8B44DEF18F0040AD8B465EF04F0C3
:10303800030AD8B459EF04F04DEF18F04DEF18F02B
:1030480082512F0AD8B486EF00F01E0AD8B44DEF8B
:1030580018F0030AD8B4A5EF00F0010AD8B4D3EFEA
:1030680001F0070AD8B44DEF18F0010AD8B44DEFB3
:1030780018F0030AD8B42BEF03F0010AD8B4FDEF17
:1030880000F00F0AD8B406EF02F04DEF18F04DEF3C
:1030980018F012003650D8B454EF18F056EF18F064
:1030A80049EF26F08DEC4DF00201EF6F2CEF26F082
:1030B800000E1B6E0B0E1A6EE8EC44F010EC51F08B
:1030C800B4C01AF0B5C01BF0E8EC44F010EC51F0B5
:1030D800B2C01AF0B3C01BF0E8EC44F010EC51F0A9
:1030E800AEC01AF0AFC01BF0E8EC44F010EC51F0A1
:1030F80010EC51F049EF26F0000E1B6E150E1A6EFB
:10310800E8EC44F010EC51F0A6C01AF01B6AE8ECA9
:1031180044F010EC51F0A7C01AF01B6AE8EC44F038
:1031280010EC51F0A8C01AF01B6AE8EC44F010EC5F
:1031380051F0A9C01AF01B6AE8EC44F010EC51F009
:10314800AAC01AF01B6AE8EC44F010EC51F0ABC0CE
:103158001AF01B6AE8EC44F010EC51F010EC51F056
:1031680049EF26F08DEC4DF0D00F0201F96F8DEC90
:103178004DF0D00F0201F86FF9510A0DF350F82500
:10318800F26F8DEC4DF0D00F0201F96F8DEC4DF020
:10319800D00F0201F86FF9510A0DF350F825F36FBB
:1031A8008DEC4DF0D00F0201F96F8DEC4DF0D00F82
:1031B8000201F86FF9510A0DF350F825F46F8DEC00
:1031C8004DF0D00F0201F96F8DEC4DF0D00F0201D8
:1031D800F86FF9510A0DF350F825F56F8DEC4DF0A5
:1031E800D00F0201F96F8DEC4DF0D00F0201F86F8E
:1031F800F9510A0DF350F825F66F8DEC4DF0D00F0C
:103208000201F96F8DEC4DF0D00F0201F86FF95102
:103218000A0DF350F825F76FF3C2DCF0F4C2DDF0C5
:10322800F5C2DEF0F6C2DFF0F7C2E0F0F25171EC61
:103238004BF0BBEC4DF0000E1B6E1F0E1A6EE8EC47
:1032480044F010EC51F0A6C01AF01B6AE8EC44F008
:1032580010EC51F0A7C01AF01B6AE8EC44F010EC2F
:1032680051F0A8C01AF01B6AE8EC44F010EC51F0D9
:10327800A9C01AF01B6AE8EC44F010EC51F0AAC09F
:103288001AF01B6AE8EC44F010EC51F0ABC01AF0ED
:103298001B6AE8EC44F010EC51F010EC51F049EFE7
:1032A80026F08DEC4DF0D00F0201F96F000E1B6E69
:1032B800290E1A6EE8EC44F010EC51F00201F951B5
:1032C800D8A469EF19F06BEF19F076EF19F0000E3A
:1032D80049EC4FF0000E1B6E000E1A6EE8EC44F03D
:1032E80081EF19F0010E49EC4FF0000E1B6E010E34
:1032F8001A6EE8EC44F081EF19F010EC51F010EC84
:1033080051F049EF26F08DEC4DF0D00F0201F96F26
:10331800000E1B6E330E1A6EE8EC44F010EC51F000
:103328000201F951D8A49BEF19F09DEF19F0A6EF0F
:1033380019F0899C000E1B6E000E1A6EE8EC44F022
:10334800ADEF19F0898C000E1B6E010E1A6EE8ECB9
:1033580044F010EC51F010EC51F049EF26F08DECF0
:103368004DF00201F06F9EEF25F08DEC4DF002015B
:10337800F16F310EF119D8A4C4EF19F0C6EF19F0A6
:10338800D1EF19F0880E146EEB0E156E010E166E45
:10339800E7EC4DF08C8849EF26F0CB0E146EEB0E5F
:1033A800156E010E166EE7EC4DF08C9849EF26F07D
:1033B80049EF26F0FF0049EF26F0140E146EED0ECB
:1033C800156E010E166EE7EC4DF02DEC2EF0C10EC9
:1033D800146EEF0E156E010E166EE7EC4DF010EC44
:1033E80051F049EF26F0250E146EED0E156E010E04
:1033F800166EE7EC4DF0F00E136E000E146E000E14
:1034080080EC4FF0C10E146EEF0E156E010E166EA5
:10341800E7EC4DF010EC51F049EF26F0EE0E146E8B
:10342800ED0E156E010E166EE7EC4DF0C1EC34F0A2
:10343800C10E146EEF0E156E010E166EE7EC4DF010
:1034480010EC51F049EF26F0F10E146E940E136E45
:10345800000EB3EC4FF00201F96FF10E146E950EE9
:10346800136E000EB3EC4FF00201F86FF851000133
:10347800E16F0201F9512A6EE1C02BF0F00E136ED4
:10348800000E146E000E80EC4FF02A4A2B2AF10E23
:10349800146E940E136E2AC015F02BC016F0000E91
:1034A8005EEC4EF0F00E146E000E136E300E166EBB
:1034B8004D0E156E000E5EEC4EF0700E146EEB0E97
:1034C800156E000E166EE7EC4DF02AC01AF02BC0F0
:1034D8001BF0E8EC44F010EC51F010EC51F049EF1F
:1034E80026F086EC50F0A90E146EEC0E156E000E48
:1034F800166EE7EC4DF0020E146E0001BA51D5ECD1
:1035080049F01B0E146EEF0E156E000E166EE7ECEA
:103518004DF0020E146E0001AC51D5EC49F010ECE0
:1035280051F010EC51F049EF26F0BE0E146EED0E7E
:10353800156E000E166EE7EC4DF0020E146E0001CB
:10354800B851D5EC49F0CE0E146EED0E156E000E86
:10355800166EE7EC4DF0020E146E0001B751D5EC73
:1035680049F0BB0E146EEC0E156E000E166EE7ECED
:103578004DF0020E146E0001B651D5EC49F0000E64
:10358800166E000E176E2F0E186EC00EA3EC4CF0C0
:10359800B60E146EEB0E156E000E166EE7EC4DF0BF
:1035A800000E0201F96F2E0EF965DDEF1AF0DFEF5C
:1035B8001AF0E3EF1AF011EF1BF011EF1BF0F9C24C
:1035C80013F0146A000E166E0A0E156E61EC46F0C2
:1035D80013501410D8A4F3EF1AF0F5EF1AF0F7EF20
:1035E8001AF010EC51F0020E146E0201F951010D9F
:1035F800C00EF324D96E020EF420DA6EDF50D5EC3B
:1036080049F00201F92B2E0EF9650DEF1BF00FEFB3
:103618001BF0E3EF1AF011EF1BF03E0E166E000ED2
:10362800176E080E186EE30EA3EC4CF0030E146E22
:10363800ED0E156E000E166EE7EC4DF0000E020151
:10364800F96F070EF9652BEF1BF02DEF1BF031EF2B
:103658001BF05DEF1BF05DEF1BF0F9C213F0146A6D
:10366800000E166E0A0E156E61EC46F0135014101B
:10367800D8A441EF1BF043EF1BF045EF1BF010EC13
:1036880051F0020E146E0201F951010DE30EF324FC
:10369800D96E000EF420DA6EDF50D5EC49F0020145
:1036A800F92B070EF9655BEF1BF05DEF1BF031EFAF
:1036B8001BF080A262EF1BF064EF1BF06EEF1BF0B3
:1036C8000A0E146EEC0E156E000E166EE7EC4DF039
:1036D80078EF1BF0A00E146EEB0E156E000E166E32
:1036E800E7EC4DF078EF1BF010EC51F010EC51F0D6
:1036F80049EF26F08DEC4DF00001946F8DEC4DF004
:103708000001956F8DEC4DF00001966F8DEC4DF03A
:103718000001986F8DEC4DF00001976F8DEC4DF026
:103728000001996FC00E136E010E146E38EC47F04D
:10373800360E146EED0E156E010E166EE7EC4DF09A
:1037480010EC51F049EF26F08DEC4DF00001946F2C
:103758008DEC4DF00001956F8DEC4DF00001966FEA
:103768008DEC4DF00001986F8DEC4DF00001976FD6
:103778008DEC4DF00001996F900E136E010E146ED2
:1037880038EC47F0580E146EED0E156E010E166EDD
:10379800E7EC4DF010EC51F049EF26F08DEC4DF0D0
:1037A8000001946F8DEC4DF00001956F8DEC4DF09C
:1037B8000001966F8DEC4DF00001986F8DEC4DF087
:1037C8000001976F8DEC4DF00001996F600E136E3C
:1037D800010E146E38EC47F07A0E146EED0E156E6D
:1037E800010E166EE7EC4DF010EC51F049EF26F0A3
:1037F8008DEC4DF00001946F8DEC4DF00001956F4C
:103808008DEC4DF00001966F8DEC4DF00001986F36
:103818008DEC4DF00001976F8DEC4DF00001996F24
:10382800900E136E020E146E38EC47F0FE0E146EF6
:10383800ED0E156E010E166EE7EC4DF010EC51F022
:1038480049EF26F08DEC4DF00001946F8DEC4DF0B2
:103858000001956F8DEC4DF00001966F8DEC4DF0E9
:103868000001986F8DEC4DF00001976F8DEC4DF0D5
:103878000001996F600E136E020E146E38EC47F05B
:103888009C0E146EED0E156E010E166EE7EC4DF0E3
:1038980010EC51F049EF26F08DEC4DF00001946FDB
:1038A8008DEC4DF00001956F8DEC4DF00001966F99
:1038B8008DEC4DF00001986F8DEC4DF00001976F85
:1038C8008DEC4DF00001996F300E136E010E146EE1
:1038D80038EC47F0470E146EED0E156E010E166E9D
:1038E800E7EC4DF010EC51F049EF26F08DEC4DF07F
:1038F8000001946F8DEC4DF00001956F8DEC4DF04B
:103908000001966F8DEC4DF00001986F8DEC4DF035
:103918000001976F8DEC4DF00001996F300E136E1A
:10392800020E146E38EC47F0690E146EED0E156E2B
:10393800010E166EE7EC4DF010EC51F049EF26F051
:103948008DEC4DF00001946F8DEC4DF00001956FFA
:103958008DEC4DF00001966F8DEC4DF00001986FE5
:103968008DEC4DF00001976F8DEC4DF00001996FD3
:10397800000E136E020E146E38EC47F08B0E146EA8
:10398800ED0E156E010E166EE7EC4DF010EC51F0D1
:1039980049EF26F08DEC4DF00001886F8DEC4DF06D
:1039A8000001896F8DEC4DF00001866F8DEC4DF0B4
:1039B8000001876F8DEC4DF00001846F8DEC4DF0A8
:1039C8000001856F8DEC4DF000018A6F8DEC4DF094
:1039D80000018B6FE00E146EEB0E156E010E166E65
:1039E800E7EC4DF010EC51F049EF26F08DEC4DF07E
:1039F8000001886F8DEC4DF00001896F8DEC4DF062
:103A08000001866F8DEC4DF00001876F8DEC4DF055
:103A18000001846F8DEC4DF00001856F8DEC4DF049
:103A280000018A6F8DEC4DF000018B6FF50E146E5E
:103A3800EB0E156E010E166EE7EC4DF010EC51F022
:103A480049EF26F08DEC4DF0286E8DEC4DF0296E87
:103A5800470E136E000E146EA5EC50F0AD0E146EEA
:103A6800ED0E156E010E166EE7EC4DF010EC51F0F0
:103A780049EF26F08DEC4DF0266E8DEC4DF0276E5B
:103A8800450E136E000E146EB4EC50F0F10E146E69
:103A9800EC0E156E010E166EE7EC4DF010EC51F0C1
:103AA80049EF26F08DEC4DF00001946F8DEC4DF050
:103AB8000001956F8DEC4DF00001966F8DEC4DF087
:103AC8000001986F8DEC4DF00001976F8DEC4DF073
:103AD8000001996F000E136E010E146E38EC47F05A
:103AE800700E146EEC0E156E010E166EE7EC4DF0AE
:103AF80010EC51F049EF26F02E0E146EEE0E156EF6
:103B0800000E166EE7EC4DF0000E0201FA6F070E7C
:103B1800FA6591EF1DF093EF1DF097EF1DF04CEF54
:103B28001EF04CEF1EF0FA51060DC00EF324D96EAC
:103B3800010EF420DA6EDF500001E16FE1511A6ED8
:103B48001B6AE8EC44F03A0E146EEE0E156E000E89
:103B5800166EE7EC4DF00201FA51060D010EF32640
:103B6800000EF422C00EF324D96E010EF420DA6E92
:103B7800DF500001E16FE1511A6E1B6AE8EC44F076
:103B88003A0E146EEE0E156E000E166EE7EC4DF042
:103B98000201FA51060D020EF326000EF422C00EA1
:103BA800F324D96E010EF420DA6EDF500001E16FC4
:103BB800E1511A6E1B6AE8EC44F03A0E146EEE0EF0
:103BC800156E000E166EE7EC4DF00201FA51060D67
:103BD800030EF326000EF422C00EF324D96E010E54
:103BE800F420DA6EDF500001E16FE1511A6E1B6AB2
:103BF800E8EC44F03A0E146EEE0E156E000E166EDA
:103C0800E7EC4DF00201FA51060D040EF326000E02
:103C1800F422C00EF324D96E010EF420DA6EDF50C0
:103C28000001E16FE1511A6E1B6AE8EC44F03A0EAC
:103C3800146EEE0E156E000E166EE7EC4DF00201D6
:103C4800FA51060D050EF326000EF422C00EF324D9
:103C5800D96E010EF420DA6EDF500001E16FE151F8
:103C68001A6E1B6AE8EC44F03A0E146EEE0E156EEE
:103C7800000E166EE7EC4DF00201FA2B070EFA65FE
:103C880048EF1EF04AEF1EF097EF1DF04CEF1EF0C4
:103C980010EC51F010EC51F049EF26F04A0E146E7A
:103CA800EE0E156E000E166EE7EC4DF0000E0201DA
:103CB800FA6F070EFA6563EF1EF065EF1EF069EF05
:103CC8001EF01EEF1FF01EEF1FF0FA51060D900EAA
:103CD800F324D96E010EF420DA6EDF500001E16F93
:103CE800E1511A6E1B6AE8EC44F03A0E146EEE0EBF
:103CF800156E000E166EE7EC4DF00201FA51060D36
:103D0800010EF326000EF422900EF324D96E010E54
:103D1800F420DA6EDF500001E16FE1511A6E1B6A80
:103D2800E8EC44F03A0E146EEE0E156E000E166EA8
:103D3800E7EC4DF00201FA51060D020EF326000ED3
:103D4800F422900EF324D96E010EF420DA6EDF50BF
:103D58000001E16FE1511A6E1B6AE8EC44F03A0E7B
:103D6800146EEE0E156E000E166EE7EC4DF00201A5
:103D7800FA51060D030EF326000EF422900EF324DA
:103D8800D96E010EF420DA6EDF500001E16FE151C7
:103D98001A6E1B6AE8EC44F03A0E146EEE0E156EBD
:103DA800000E166EE7EC4DF00201FA51060D040EF6
:103DB800F326000EF422900EF324D96E010EF4209F
:103DC800DA6EDF500001E16FE1511A6E1B6AE8EC10
:103DD80044F03A0E146EEE0E156E000E166EE7ECF9
:103DE8004DF00201FA51060D050EF326000EF422DD
:103DF800900EF324D96E010EF420DA6EDF50000124
:103E0800E16FE1511A6E1B6AE8EC44F03A0E146E49
:103E1800EE0E156E000E166EE7EC4DF00201FA2B51
:103E2800070EFA651AEF1FF01CEF1FF069EF1EF07E
:103E38001EEF1FF010EC51F010EC51F049EF26F096
:103E4800660E146EEE0E156E000E166EE7EC4DF053
:103E5800000E0201FA6F070EFA6535EF1FF037EF13
:103E68001FF03BEF1FF0F0EF1FF0F0EF1FF0FA51DB
:103E7800060D600EF324D96E010EF420DA6EDF50C1
:103E88000001E16FE1511A6E1B6AE8EC44F03A0E4A
:103E9800146EEE0E156E000E166EE7EC4DF0020174
:103EA800FA51060D010EF326000EF422600EF324DB
:103EB800D96E010EF420DA6EDF500001E16FE15196
:103EC8001A6E1B6AE8EC44F03A0E146EEE0E156E8C
:103ED800000E166EE7EC4DF00201FA51060D020EC7
:103EE800F326000EF422600EF324D96E010EF4209E
:103EF800DA6EDF500001E16FE1511A6E1B6AE8ECDF
:103F080044F03A0E146EEE0E156E000E166EE7ECC7
:103F18004DF00201FA51060D030EF326000EF422AD
:103F2800600EF324D96E010EF420DA6EDF50000122
:103F3800E16FE1511A6E1B6AE8EC44F03A0E146E18
:103F4800EE0E156E000E166EE7EC4DF00201FA51FA
:103F5800060D040EF326000EF422600EF324D96E2B
:103F6800010EF420DA6EDF500001E16FE1511A6EA4
:103F78001B6AE8EC44F03A0E146EEE0E156E000E55
:103F8800166EE7EC4DF00201FA51060D050EF32608
:103F9800000EF422600EF324D96E010EF420DA6EBE
:103FA800DF500001E16FE1511A6E1B6AE8EC44F042
:103FB8003A0E146EEE0E156E000E166EE7EC4DF00E
:103FC8000201FA2B070EFA65ECEF1FF0EEEF1FF077
:103FD8003BEF1FF0F0EF1FF010EC51F010EC51F038
:103FE80049EF26F00E0E146EEF0E156E000E166ECB
:103FF800E7EC4DF0000E0201FA6F070EFA6507EFC5
:1040080020F009EF20F00DEF20F0C2EF20F0C2EF12
:1040180020F0FA51060D900EF324D96E020EF4200A
:10402800DA6EDF500001E16FE1511A6E1B6AE8ECAD
:1040380044F03A0E146EEE0E156E000E166EE7EC96
:104048004DF00201FA51060D010EF326000EF4227E
:10405800900EF324D96E020EF420DA6EDF500001C0
:10406800E16FE1511A6E1B6AE8EC44F03A0E146EE7
:10407800EE0E156E000E166EE7EC4DF00201FA51C9
:10408800060D020EF326000EF422900EF324D96ECC
:10409800020EF420DA6EDF500001E16FE1511A6E72
:1040A8001B6AE8EC44F03A0E146EEE0E156E000E24
:1040B800166EE7EC4DF00201FA51060D030EF326D9
:1040C800000EF422900EF324D96E020EF420DA6E5C
:1040D800DF500001E16FE1511A6E1B6AE8EC44F011
:1040E8003A0E146EEE0E156E000E166EE7EC4DF0DD
:1040F8000201FA51060D040EF326000EF422900E6A
:10410800F324D96E020EF420DA6EDF500001E16F5D
:10411800E1511A6E1B6AE8EC44F03A0E146EEE0E8A
:10412800156E000E166EE7EC4DF00201FA51060D01
:10413800050EF326000EF422900EF324D96E020E1B
:10414800F420DA6EDF500001E16FE1511A6E1B6A4C
:10415800E8EC44F03A0E146EEE0E156E000E166E74
:10416800E7EC4DF00201FA2B070EFA65BEEF20F0DE
:10417800C0EF20F00DEF20F0C2EF20F010EC51F06E
:1041880010EC51F049EF26F0820E146EEE0E156E0B
:10419800000E166EE7EC4DF0000E0201FA6F070EE6
:1041A800FA65D9EF20F0DBEF20F0DFEF20F094EF95
:1041B80021F094EF21F0FA51060D600EF324D96E28
:1041C800020EF420DA6EDF500001E16FE1511A6E41
:1041D8001B6AE8EC44F03A0E146EEE0E156E000EF3
:1041E800166EE7EC4DF00201FA51060D010EF326AA
:1041F800000EF422600EF324D96E020EF420DA6E5B
:10420800DF500001E16FE1511A6E1B6AE8EC44F0DF
:104218003A0E146EEE0E156E000E166EE7EC4DF0AB
:104228000201FA51060D020EF326000EF422600E6A
:10423800F324D96E020EF420DA6EDF500001E16F2C
:10424800E1511A6E1B6AE8EC44F03A0E146EEE0E59
:10425800156E000E166EE7EC4DF00201FA51060DD0
:10426800030EF326000EF422600EF324D96E020E1C
:10427800F420DA6EDF500001E16FE1511A6E1B6A1B
:10428800E8EC44F03A0E146EEE0E156E000E166E43
:10429800E7EC4DF00201FA51060D040EF326000E6C
:1042A800F422600EF324D96E020EF420DA6EDF5089
:1042B8000001E16FE1511A6E1B6AE8EC44F03A0E16
:1042C800146EEE0E156E000E166EE7EC4DF0020140
:1042D800FA51060D050EF326000EF422600EF324A3
:1042E800D96E020EF420DA6EDF500001E16FE15161
:1042F8001A6E1B6AE8EC44F03A0E146EEE0E156E58
:10430800000E166EE7EC4DF00201FA2B070EFA6567
:1043180090EF21F092EF21F0DFEF20F094EF21F001
:1043280010EC51F010EC51F049EF26F03C0E146EF1
:10433800EE0E156E000E166EE7EC4DF0000E020143
:10434800FA6F070EFA65ABEF21F0ADEF21F0B1EF90
:1043580021F066EF22F066EF22F0FA51060D300EDA
:10436800F324D96E010EF420DA6EDF500001E16FFC
:10437800E1511A6E1B6AE8EC44F03A0E146EEE0E28
:10438800156E000E166EE7EC4DF00201FA51060D9F
:10439800010EF326000EF422300EF324D96E010E1E
:1043A800F420DA6EDF500001E16FE1511A6E1B6AEA
:1043B800E8EC44F03A0E146EEE0E156E000E166E12
:1043C800E7EC4DF00201FA51060D020EF326000E3D
:1043D800F422300EF324D96E010EF420DA6EDF5089
:1043E8000001E16FE1511A6E1B6AE8EC44F03A0EE5
:1043F800146EEE0E156E000E166EE7EC4DF002010F
:10440800FA51060D030EF326000EF422300EF324A3
:10441800D96E010EF420DA6EDF500001E16FE15130
:104428001A6E1B6AE8EC44F03A0E146EEE0E156E26
:10443800000E166EE7EC4DF00201FA51060D040E5F
:10444800F326000EF422300EF324D96E010EF42068
:10445800DA6EDF500001E16FE1511A6E1B6AE8EC79
:1044680044F03A0E146EEE0E156E000E166EE7EC62
:104478004DF00201FA51060D050EF326000EF42246
:10448800300EF324D96E010EF420DA6EDF500001ED
:10449800E16FE1511A6E1B6AE8EC44F03A0E146EB3
:1044A800EE0E156E000E166EE7EC4DF00201FA2BBB
:1044B800070EFA6562EF22F064EF22F0B1EF21F007
:1044C80066EF22F010EC51F010EC51F049EF26F0B5
:1044D800580E146EEE0E156E000E166EE7EC4DF0CB
:1044E800000E0201FA6F070EFA657DEF22F07FEFEA
:1044F80022F083EF22F038EF23F038EF23F0FA515F
:10450800060D300EF324D96E020EF420DA6EDF5059
:104518000001E16FE1511A6E1B6AE8EC44F03A0EB3
:10452800146EEE0E156E000E166EE7EC4DF00201DD
:10453800FA51060D010EF326000EF422300EF32474
:10454800D96E020EF420DA6EDF500001E16FE151FE
:104558001A6E1B6AE8EC44F03A0E146EEE0E156EF5
:10456800000E166EE7EC4DF00201FA51060D020E30
:10457800F326000EF422300EF324D96E020EF42036
:10458800DA6EDF500001E16FE1511A6E1B6AE8EC48
:1045980044F03A0E146EEE0E156E000E166EE7EC31
:1045A8004DF00201FA51060D030EF326000EF42217
:1045B800300EF324D96E020EF420DA6EDF500001BB
:1045C800E16FE1511A6E1B6AE8EC44F03A0E146E82
:1045D800EE0E156E000E166EE7EC4DF00201FA5164
:1045E800060D040EF326000EF422300EF324D96EC5
:1045F800020EF420DA6EDF500001E16FE1511A6E0D
:104608001B6AE8EC44F03A0E146EEE0E156E000EBE
:10461800166EE7EC4DF00201FA51060D050EF32671
:10462800000EF422300EF324D96E020EF420DA6E56
:10463800DF500001E16FE1511A6E1B6AE8EC44F0AB
:104648003A0E146EEE0E156E000E166EE7EC4DF077
:104658000201FA2B070EFA6534EF23F036EF23F048
:1046680083EF22F038EF23F010EC51F010EC51F00A
:1046780049EF26F0740E146EEE0E156E000E166ECF
:10468800E7EC4DF0000E0201FA6F070EFA654FEFE6
:1046980023F051EF23F055EF23F00AEF24F00AEF4F
:1046A80024F0FA51060D000EF324D96E020EF42000
:1046B800DA6EDF500001E16FE1511A6E1B6AE8EC17
:1046C80044F03A0E146EEE0E156E000E166EE7EC00
:1046D8004DF00201FA51060D010EF326000EF422E8
:1046E800000EF324D96E020EF420DA6EDF500001BA
:1046F800E16FE1511A6E1B6AE8EC44F03A0E146E51
:10470800EE0E156E000E166EE7EC4DF00201FA5132
:10471800060D020EF326000EF422000EF324D96EC5
:10472800020EF420DA6EDF500001E16FE1511A6EDB
:104738001B6AE8EC44F03A0E146EEE0E156E000E8D
:10474800166EE7EC4DF00201FA51060D030EF32642
:10475800000EF422000EF324D96E020EF420DA6E55
:10476800DF500001E16FE1511A6E1B6AE8EC44F07A
:104778003A0E146EEE0E156E000E166EE7EC4DF046
:104788000201FA51060D040EF326000EF422000E63
:10479800F324D96E020EF420DA6EDF500001E16FC7
:1047A800E1511A6E1B6AE8EC44F03A0E146EEE0EF4
:1047B800156E000E166EE7EC4DF00201FA51060D6B
:1047C800050EF326000EF422000EF324D96E020E15
:1047D800F420DA6EDF500001E16FE1511A6E1B6AB6
:1047E800E8EC44F03A0E146EEE0E156E000E166EDE
:1047F800E7EC4DF00201FA2B070EFA6506EF24F0FC
:1048080008EF24F055EF23F00AEF24F010EC51F0F4
:1048180010EC51F049EF26F0CD0E146EEC0E156E2B
:10482800010E166EE7EC4DF088C01AF01B6AE8EC32
:1048380044F03A0E146EEE0E156E000E166EE7EC8E
:104848004DF089C01AF01B6AE8EC44F010EC51F006
:1048580086C01AF01B6AE8EC44F03A0E146EEE0EAD
:10486800156E000E166EE7EC4DF087C01AF01B6A45
:10487800E8EC44F010EC51F084C01AF01B6AE8EC44
:1048880044F03A0E146EEE0E156E000E166EE7EC3E
:104898004DF085C01AF01B6AE8EC44F010EC51F0BA
:1048A8008AC01AF01B6AE8EC44F03A0E146EEE0E59
:1048B800156E000E166EE7EC4DF08BC01AF01B6AF1
:1048C800E8EC44F010EC51F049EF26F0DF0E146EDE
:1048D800EC0E156E010E166EE7EC4DF088C01AF05E
:1048E8001B6AE8EC44F089C01AF01B6AE8EC44F053
:1048F80086C01AF01B6AE8EC44F087C01AF01B6AFD
:10490800E8EC44F084C01AF01B6AE8EC44F085C077
:104918001AF01B6AE8EC44F08AC01AF01B6AE8EC4B
:1049280044F08BC01AF01B6AE8EC44F010EC51F02C
:1049380049EF26F0CD0E146EEC0E156E010E166EB4
:10494800E7EC4DF028C01AF01B6AE8EC44F029C0E7
:104958001AF01B6AE8EC44F010EC51F049EF26F02D
:10496800CD0E146EEC0E156E010E166EE7EC4DF0C2
:1049780026C01AF01B6AE8EC44F027C01AF01B6A3C
:10498800E8EC44F010EC51F049EF26F0DE0E146E1E
:10499800ED0E156E010E166EE7EC4DF0000E0201DD
:1049A800FA6F070EFA65DBEF24F0DDEF24F0E1EF94
:1049B80024F096EF25F096EF25F0FA51060D000E3B
:1049C800F324D96E010EF420DA6EDF500001E16F96
:1049D800E1511A6E1B6AE8EC44F03A0E146EEE0EC2
:1049E800156E000E166EE7EC4DF00201FA51060D39
:1049F800010EF326000EF422000EF324D96E010EE8
:104A0800F420DA6EDF500001E16FE1511A6E1B6A83
:104A1800E8EC44F03A0E146EEE0E156E000E166EAB
:104A2800E7EC4DF00201FA51060D020EF326000ED6
:104A3800F422000EF324D96E010EF420DA6EDF5052
:104A48000001E16FE1511A6E1B6AE8EC44F03A0E7E
:104A5800146EEE0E156E000E166EE7EC4DF00201A8
:104A6800FA51060D030EF326000EF422000EF3246D
:104A7800D96E010EF420DA6EDF500001E16FE151CA
:104A88001A6E1B6AE8EC44F03A0E146EEE0E156EC0
:104A9800000E166EE7EC4DF00201FA51060D040EF9
:104AA800F326000EF422000EF324D96E010EF42032
:104AB800DA6EDF500001E16FE1511A6E1B6AE8EC13
:104AC80044F03A0E146EEE0E156E000E166EE7ECFC
:104AD8004DF00201FA51060D050EF326000EF422E0
:104AE800000EF324D96E010EF420DA6EDF500001B7
:104AF800E16FE1511A6E1B6AE8EC44F03A0E146E4D
:104B0800EE0E156E000E166EE7EC4DF00201FA2B54
:104B1800070EFA6592EF25F094EF25F0E1EF24F007
:104B280096EF25F010EC51F010EC51F049EF26F01B
:104B380049EF26F00201F051410AD8B480EF1DF088
:104B4800030AD8B452EF1EF0010AD8B424EF1FF0BC
:104B5800070AD8B4F6EF1FF0010AD8B4C8EF20F05E
:104B6800030AD8B49AEF21F0010AD8B46CEF22F006
:104B78000F0AD8B43EEF23F0010AD8B410EF24F09E
:104B8800030AD8B46AEF24F0010AD8B49EEF24F0DF
:104B9800070AD8B4B4EF24F0010AD8B475EF1AF0B4
:104BA800030AD8B4CAEF24F0010AD8B4E1EF19F027
:104BB8001E0AD8B4B9EF19F0030AD8B4F7EF19F000
:104BC800010AD8B412EF1AF0070AD8B428EF1AF07D
:104BD800030AD8B499EF1AF00D0AD8B4DEEF19F029
:104BE8003B0AD8B47EEF1BF0030AD8B4A8EF1BF039
:104BF800010AD8B4D2EF1BF0070AD8B4FCEF1BF0B7
:104C0800010AD8B426EF1CF0030AD8B450EF1CF000
:104C1800010AD8B47AEF1CF00F0AD8B4A4EF1CF03C
:104C2800010AD8B4CEEF1CF0030AD8B4FAEF1CF08E
:104C3800010AD8B426EF1DF0070AD8B43EEF1DF0DC
:104C4800020AD8B456EF1DF049EF26F049EF26F0D6
:104C5800EF51310AD8B45CEF18F0030AD8B480EFEA
:104C680018F0010AD8B4B6EF18F0070AD8B455EF0F
:104C780019F0010AD8B487EF19F0030AD8B4B3EFD2
:104C880019F049EF26F049EF26F01200899400F058
:104C980000F000F000F000F000F000F000F000F08C
:104CA80000F000F000F000F000F000F000F000F07C
:104CB80000F000F000F000F000F000F000F000F06C
:104CC80000F000F000F000F000F000F000F000F05C
:1054580000F000F000F000F000F000F000F08984A7
:1054680000F000F000F000F000F000F000F000F0B4
:1054780000F000F000F000F000F000F000F000F0A4
:1054880000F000F000F000F000F000F000F000F094
:1054980000F000F000F000F000F000F000F000F084
:105C380089941FEF2EF084B024EF2EF026EF2EF07B
:105C48001FEF2EF028EF2EF0300E31EC4DF0898446
:105C58001200000E1D6E070E1D6435EF2EF037EF93
:105C68002EF03BEF2EF0D2EF2EF0D2EF2EF01D509B
:105C7800060DC00EF324D96E010EF420DA6E1D5005
:105C8800060D000EF324136EF00EF420146E000EB1
:105C9800B3EC4FF0DF6E1D50060D010EF326000E1B
:105CA800F422C00EF324D96E010EF420DA6E1D50D2
:105CB800060D010EF324136EF00EF420146E000E80
:105CC800B3EC4FF0DF6E1D50060D020EF326000EEA
:105CD800F422C00EF324D96E010EF420DA6E1D50A2
:105CE800060D020EF324136EF00EF420146E000E4F
:105CF800B3EC4FF0DF6E1D50060D040EF326000EB8
:105D0800F422C00EF324D96E010EF420DA6E1D5071
:105D1800060D030EF324136EF00EF420146E000E1D
:105D2800B3EC4FF0DF6E1D50060D030EF326000E88
:105D3800F422C00EF324D96E010EF420DA6E1D5041
:105D4800060D040EF324136EF00EF420146E000EEC
:105D5800B3EC4FF0DF6E1D50060D050EF326000E56
:105D6800F422C00EF324D96E010EF420DA6E1D5011
:105D7800060D050EF324136EF00EF420146E000EBB
:105D8800B3EC4FF0DF6E1D2A070E1D64CEEF2EF028
:105D9800D0EF2EF03BEF2EF0D2EF2EF0000E1D6E5E
:105DA800070E1D64DAEF2EF0DCEF2EF0E0EF2EF098
:105DB80077EF2FF077EF2FF01D50060D900EF3249C
:105DC800D96E010EF420DA6E1D50060D300EF32444
:105DD800136EF00EF420146E000EB3EC4FF0DF6E6D
:105DE8001D50060D010EF326000EF422900EF3242A
:105DF800D96E010EF420DA6E1D50060D310EF32413
:105E0800136EF00EF420146E000EB3EC4FF0DF6E3C
:105E18001D50060D020EF326000EF422900EF324F8
:105E2800D96E010EF420DA6E1D50060D320EF324E1
:105E3800136EF00EF420146E000EB3EC4FF0DF6E0C
:105E48001D50060D040EF326000EF422900EF324C6
:105E5800D96E010EF420DA6E1D50060D330EF324B0
:105E6800136EF00EF420146E000EB3EC4FF0DF6EDC
:105E78001D50060D030EF326000EF422900EF32497
:105E8800D96E010EF420DA6E1D50060D340EF3247F
:105E9800136EF00EF420146E000EB3EC4FF0DF6EAC
:105EA8001D50060D050EF326000EF422900EF32465
:105EB800D96E010EF420DA6E1D50060D350EF3244E
:105EC800136EF00EF420146E000EB3EC4FF0DF6E7C
:105ED8001D2A070E1D6473EF2FF075EF2FF0E0EF0A
:105EE8002EF077EF2FF0000E1D6E070E1D647FEF6A
:105EF8002FF081EF2FF085EF2FF01CEF30F01CEF23
:105F080030F01D50060D600EF324D96E010EF420FA
:105F1800DA6E1D50060D600EF324136EF00EF42099
:105F2800146E000EB3EC4FF0DF6E1D50060D010E1F
:105F3800F326000EF422600EF324D96E010EF4202D
:105F4800DA6E1D50060D610EF324136EF00EF42068
:105F5800146E000EB3EC4FF0DF6E1D50060D020EEE
:105F6800F326000EF422600EF324D96E010EF420FD
:105F7800DA6E1D50060D620EF324136EF00EF42037
:105F8800146E000EB3EC4FF0DF6E1D50060D040EBC
:105F9800F326000EF422600EF324D96E010EF420CD
:105FA800DA6E1D50060D630EF324136EF00EF42006
:105FB800146E000EB3EC4FF0DF6E1D50060D030E8D
:105FC800F326000EF422600EF324D96E010EF4209D
:105FD800DA6E1D50060D640EF324136EF00EF420D5
:105FE800146E000EB3EC4FF0DF6E1D50060D050E5B
:105FF800F326000EF422600EF324D96E010EF4206D
:10600800DA6E1D50060D650EF324136EF00EF420A3
:10601800146E000EB3EC4FF0DF6E1D2A070E1D64E0
:1060280018EF30F01AEF30F085EF2FF01CEF30F05A
:10603800000E1D6E070E1D6424EF30F026EF30F0C1
:106048002AEF30F0C1EF30F0C1EF30F01D50060DEF
:10605800900EF324D96E020EF420DA6E1D50060D50
:10606800900EF324136EF00EF420146E000EB3ECB1
:106078004FF0DF6E1D50060D010EF326000EF422C0
:10608800900EF324D96E020EF420DA6E1D50060D20
:10609800910EF324136EF00EF420146E000EB3EC80
:1060A8004FF0DF6E1D50060D020EF326000EF4228F
:1060B800900EF324D96E020EF420DA6E1D50060DF0
:1060C800920EF324136EF00EF420146E000EB3EC4F
:1060D8004FF0DF6E1D50060D040EF326000EF4225D
:1060E800900EF324D96E020EF420DA6E1D50060DC0
:1060F800930EF324136EF00EF420146E000EB3EC1E
:106108004FF0DF6E1D50060D030EF326000EF4222D
:10611800900EF324D96E020EF420DA6E1D50060D8F
:10612800940EF324136EF00EF420146E000EB3ECEC
:106138004FF0DF6E1D50060D050EF326000EF422FB
:10614800900EF324D96E020EF420DA6E1D50060D5F
:10615800950EF324136EF00EF420146E000EB3ECBB
:106168004FF0DF6E1D2A070E1D64BDEF30F0BFEF44
:1061780030F02AEF30F0C1EF30F0000E1D6E070E40
:106188001D64C9EF30F0CBEF30F0CFEF30F066EFA1
:1061980031F066EF31F01D50060D600EF324D96E14
:1061A800020EF420DA6E1D50060DC00EF324136E95
:1061B800F00EF420146E000EB3EC4FF0DF6E1D509D
:1061C800060D010EF326000EF422600EF324D96E9C
:1061D800020EF420DA6E1D50060DC10EF324136E64
:1061E800F00EF420146E000EB3EC4FF0DF6E1D506D
:1061F800060D020EF326000EF422600EF324D96E6B
:10620800020EF420DA6E1D50060DC20EF324136E32
:10621800F00EF420146E000EB3EC4FF0DF6E1D503C
:10622800060D040EF326000EF422600EF324D96E38
:10623800020EF420DA6E1D50060DC30EF324136E01
:10624800F00EF420146E000EB3EC4FF0DF6E1D500C
:10625800060D030EF326000EF422600EF324D96E09
:10626800020EF420DA6E1D50060DC40EF324136ED0
:10627800F00EF420146E000EB3EC4FF0DF6E1D50DC
:10628800060D050EF326000EF422600EF324D96ED7
:10629800020EF420DA6E1D50060DC50EF324136E9F
:1062A800F00EF420146E000EB3EC4FF0DF6E1D2AD2
:1062B800070E1D6462EF31F064EF31F0CFEF30F07C
:1062C80066EF31F0000E1D6E070E1D646EEF31F0A3
:1062D80070EF31F074EF31F00BEF32F00BEF32F07A
:1062E8001D50060D300EF324D96E010EF420DA6E1F
:1062F8001D50060DF00EF324136EF00EF420146EEC
:10630800000EB3EC4FF0DF6E1D50060D010EF326A4
:10631800000EF422300EF324D96E010EF420DA6E4A
:106328001D50060DF10EF324136EF00EF420146EBA
:10633800000EB3EC4FF0DF6E1D50060D020EF32673
:10634800000EF422300EF324D96E010EF420DA6E1A
:106358001D50060DF20EF324136EF00EF420146E89
:10636800000EB3EC4FF0DF6E1D50060D040EF32641
:10637800000EF422300EF324D96E010EF420DA6EEA
:106388001D50060DF30EF324136EF00EF420146E58
:10639800000EB3EC4FF0DF6E1D50060D030EF32612
:1063A800000EF422300EF324D96E010EF420DA6EBA
:1063B8001D50060DF40EF324136EF00EF420146E27
:1063C800000EB3EC4FF0DF6E1D50060D050EF326E0
:1063D800000EF422300EF324D96E010EF420DA6E8A
:1063E8001D50060DF50EF324136EF00EF420146EF6
:1063F800000EB3EC4FF0DF6E1D2A070E1D6407EF89
:1064080032F009EF32F074EF31F00BEF32F0000E9A
:106418001D6E070E1D6413EF32F015EF32F019EF01
:1064280032F0B0EF32F0B0EF32F01D50060D300E02
:10643800F324D96E020EF420DA6E1D50060D200EDC
:10644800F324136EF10EF420146E000EB3EC4FF02B
:10645800DF6E1D50060D010EF326000EF422300EDD
:10646800F324D96E020EF420DA6E1D50060D210EAB
:10647800F324136EF10EF420146E000EB3EC4FF0FB
:10648800DF6E1D50060D020EF326000EF422300EAC
:10649800F324D96E020EF420DA6E1D50060D220E7A
:1064A800F324136EF10EF420146E000EB3EC4FF0CB
:1064B800DF6E1D50060D040EF326000EF422300E7A
:1064C800F324D96E020EF420DA6E1D50060D230E49
:1064D800F324136EF10EF420146E000EB3EC4FF09B
:1064E800DF6E1D50060D030EF326000EF422300E4B
:1064F800F324D96E020EF420DA6E1D50060D240E18
:10650800F324136EF10EF420146E000EB3EC4FF06A
:10651800DF6E1D50060D050EF326000EF422300E18
:10652800F324D96E020EF420DA6E1D50060D250EE6
:10653800F324136EF10EF420146E000EB3EC4FF03A
:10654800DF6E1D2A070E1D64ACEF32F0AEEF32F09D
:1065580019EF32F0B0EF32F0000E1D6E070E1D6419
:10656800B8EF32F0BAEF32F0BEEF32F055EF33F059
:1065780055EF33F01D50060D000EF324D96E020EB0
:10658800F420DA6E1D50060D500EF324136EF10E32
:10659800F420146E000EB3EC4FF0DF6E1D50060DA4
:1065A800010EF326000EF422000EF324D96E020E1B
:1065B800F420DA6E1D50060D510EF324136EF10E01
:1065C800F420146E000EB3EC4FF0DF6E1D50060D74
:1065D800020EF326000EF422000EF324D96E020EEA
:1065E800F420DA6E1D50060D520EF324136EF10ED0
:1065F800F420146E000EB3EC4FF0DF6E1D50060D44
:10660800040EF326000EF422000EF324D96E020EB7
:10661800F420DA6E1D50060D530EF324136EF10E9E
:10662800F420146E000EB3EC4FF0DF6E1D50060D13
:10663800030EF326000EF422000EF324D96E020E88
:10664800F420DA6E1D50060D540EF324136EF10E6D
:10665800F420146E000EB3EC4FF0DF6E1D50060DE3
:10666800050EF326000EF422000EF324D96E020E56
:10667800F420DA6E1D50060D550EF324136EF10E3C
:10668800F420146E000EB3EC4FF0DF6E1D2A070ED7
:106698001D6451EF33F053EF33F0BEEF32F055EF96
:1066A80033F0F10E146E800E136E000EB3EC4FF043
:1066B8000001BF6FF10E146E810E136E000EB3EC65
:1066C8004FF00001C06FF10E146E820E136E000EB3
:1066D800B3EC4FF00001C16FF10E146E830E136E10
:1066E800000EB3EC4FF00001C26FF10E146E840E71
:1066F800136E000EB3EC4FF00001C36FF10E146E71
:10670800850E136E000EB3EC4FF00001C46FF10E4E
:10671800146E860E136E000EB3EC4FF00001C56FB9
:10672800F10E146E870E136E000EB3EC4FF00001DD
:10673800C66FF10E146E890E136E000EB3EC4FF097
:1067480000018C6FF10E146E8A0E136E000EB3ECFE
:106758004FF000018D6FF10E146E8B0E136E000E4C
:10676800B3EC4FF000018E6FF10E146E8C0E136EA9
:10677800000EB3EC4FF000018F6FF10E146E8D0E0A
:10678800136E000EB3EC4FF00001906FF10E146E13
:106798008E0E136E000EB3EC4FF00001916FF10EE8
:1067A800146E8F0E136E000EB3EC4FF00001926F53
:1067B800F10E146E900E136E000EB3EC4FF0000144
:1067C800936FF10E146E900E136E000EB3EC4FF033
:1067D800476EF10E146E910E136E000EB3EC4FF06F
:1067E800486EF10E146E920E136E000EB3EC4FF05D
:1067F800456EF10E146E930E136E000EB3EC4FF04F
:10680800466EF10E146E940E136E000EB3EC4FF03C
:106818001B6EF10E146E950E136E000EB3EC4FF056
:106828001C6E1C50196E1B502A6E19C02BF0000EDE
:106838001D6E070E1D6423EF34F025EF34F029EFA9
:1068480034F0C0EF34F0C0EF34F01D50060D000EE8
:10685800F324D96E010EF420DA6E1D50060D960E43
:10686800F324136EF10EF420146E000EB3EC4FF007
:10687800DF6E1D50060D010EF326000EF422000EE9
:10688800F324D96E010EF420DA6E1D50060D970E12
:10689800F324136EF10EF420146E000EB3EC4FF0D7
:1068A800DF6E1D50060D020EF326000EF422000EB8
:1068B800F324D96E010EF420DA6E1D50060D980EE1
:1068C800F324136EF10EF420146E000EB3EC4FF0A7
:1068D800DF6E1D50060D040EF326000EF422000E86
:1068E800F324D96E010EF420DA6E1D50060D990EB0
:1068F800F324136EF10EF420146E000EB3EC4FF077
:10690800DF6E1D50060D030EF326000EF422000E56
:10691800F324D96E010EF420DA6E1D50060D9A0E7E
:10692800F324136EF10EF420146E000EB3EC4FF046
:10693800DF6E1D50060D050EF326000EF422000E24
:10694800F324D96E010EF420DA6E1D50060D9B0E4D
:10695800F324136EF10EF420146E000EB3EC4FF016
:10696800DF6E1D2A070E1D64BCEF34F0BEEF34F055
:1069780029EF34F0C0EF34F01200000E1F6E070E3E
:106988001F64C9EF34F0CBEF34F0CFEF34F063EF8E
:1069980035F063EF35F01F50060DC00EF324D96EA5
:1069A800010EF420DA6EDF501A6E1F50060D010E2C
:1069B800F326000EF422C00EF324D96E010EF42043
:1069C800DA6EDF501B6E1A501D6E1BC01EF01F5072
:1069D800060D000EF324136EF00EF420146E1DC085
:1069E80015F01EC016F0000E5EEC4EF01F50060D9E
:1069F800020EF326000EF422C00EF324D96E010E07
:106A0800F420DA6EDF501A6E1F50060D040EF326BE
:106A1800000EF422C00EF324D96E010EF420DA6EB3
:106A2800DF501B6E1A501D6E1BC01EF01F50060D46
:106A3800020EF324136EF00EF420146E1DC015F030
:106A48001EC016F0000E5EEC4EF01F50060D030E31
:106A5800F326000EF422C00EF324D96E010EF420A2
:106A6800DA6EDF501A6E1F50060D050EF326000E63
:106A7800F422C00EF324D96E010EF420DA6EDF5032
:106A88001B6E1A501D6E1BC01EF01F50060D040E03
:106A9800F324136EF00EF420146E1DC015F01EC002
:106AA80016F0000E5EEC4EF01F2A070E1F645FEF13
:106AB80035F061EF35F0CFEF34F063EF35F0000ECD
:106AC8001F6E070E1F646BEF35F06DEF35F071EF39
:106AD80035F005EF36F005EF36F01F50060D900E35
:106AE800F324D96E010EF420DA6EDF501A6E1F50AF
:106AF800060D010EF326000EF422900EF324D96E33
:106B0800010EF420DA6EDF501B6E1A501D6E1BC08A
:106B18001EF01F50060D300EF324136EF00EF420F5
:106B2800146E1DC015F01EC016F0000E5EEC4EF07F
:106B38001F50060D020EF326000EF422900EF324C9
:106B4800D96E010EF420DA6EDF501A6E1F50060D52
:106B5800040EF326000EF422900EF324D96E010ED3
:106B6800F420DA6EDF501B6E1A501D6E1BC01EF02B
:106B78001F50060D320EF324136EF00EF420146E1F
:106B88001DC015F01EC016F0000E5EEC4EF01F5032
:106B9800060D030EF326000EF422900EF324D96E90
:106BA800010EF420DA6EDF501A6E1F50060D050E26
:106BB800F326000EF422900EF324D96E010EF42071
:106BC800DA6EDF501B6E1A501D6E1BC01EF01F5070
:106BD800060D340EF324136EF00EF420146E1DC04F
:106BE80015F01EC016F0000E5EEC4EF01F2A070EC0
:106BF8001F6401EF36F003EF36F071EF35F005EF63
:106C080036F0000E1F6E070E1F640DEF36F00FEF03
:106C180036F013EF36F0A7EF36F0A7EF36F01F5037
:106C2800060D600EF324D96E010EF420DA6EDF50E3
:106C38001A6E1F50060D010EF326000EF422600E88
:106C4800F324D96E010EF420DA6EDF501B6E1A5051
:106C58001D6E1BC01EF01F50060D600EF324136E30
:106C6800F00EF420146E1DC015F01EC016F0000EB4
:106C78005EEC4EF01F50060D020EF326000EF422B5
:106C8800600EF324D96E010EF420DA6EDF501A6E0E
:106C98001F50060D040EF326000EF422600EF32496
:106CA800D96E010EF420DA6EDF501B6E1A501D6E7D
:106CB8001BC01EF01F50060D620EF324136EF00E5B
:106CC800F420146E1DC015F01EC016F0000E5EEC08
:106CD8004EF01F50060D030EF326000EF422600E30
:106CE800F324D96E010EF420DA6EDF501A6E1F50AD
:106CF800060D050EF326000EF422600EF324D96E5D
:106D0800010EF420DA6EDF501B6E1A501D6E1BC088
:106D18001EF01F50060D640EF324136EF00EF420BF
:106D2800146E1DC015F01EC016F0000E5EEC4EF07D
:106D38001F2A070E1F64A3EF36F0A5EF36F013EFF6
:106D480036F0A7EF36F0000E1F6E070E1F64AFEF88
:106D580036F0B1EF36F0B5EF36F049EF37F049EFDE
:106D680037F01F50060D900EF324D96E020EF42052
:106D7800DA6EDF501A6E1F50060D010EF326000E54
:106D8800F422900EF324D96E020EF420DA6EDF504E
:106D98001B6E1A501D6E1BC01EF01F50060D900E64
:106DA800F324136EF00EF420146E1DC015F01EC0EF
:106DB80016F0000E5EEC4EF01F50060D020EF32684
:106DC800000EF422900EF324D96E020EF420DA6E2F
:106DD800DF501A6E1F50060D040EF326000EF42223
:106DE800900EF324D96E020EF420DA6EDF501B6E7B
:106DF8001A501D6E1BC01EF01F50060D920EF32474
:106E0800136EF00EF420146E1DC015F01EC016F09F
:106E1800000E5EEC4EF01F50060D030EF326000E1A
:106E2800F422900EF324D96E020EF420DA6EDF50AD
:106E38001A6E1F50060D050EF326000EF422900E52
:106E4800F324D96E020EF420DA6EDF501B6E1A504E
:106E58001D6E1BC01EF01F50060D940EF324136EFA
:106E6800F00EF420146E1DC015F01EC016F0000EB2
:106E78005EEC4EF01F2A070E1F6445EF37F047EF10
:106E880037F0B5EF36F049EF37F0000E1F6E070EFA
:106E98001F6451EF37F053EF37F057EF37F0EBEF50
:106EA80037F0EBEF37F01F50060D600EF324D96E64
:106EB800020EF420DA6EDF501A6E1F50060D010E16
:106EC800F326000EF422600EF324D96E020EF4208D
:106ED800DA6EDF501B6E1A501D6E1BC01EF01F505D
:106EE800060DC00EF324136EF00EF420146E1DC0B0
:106EF80015F01EC016F0000E5EEC4EF01F50060D89
:106F0800020EF326000EF422600EF324D96E020E50
:106F1800F420DA6EDF501A6E1F50060D040EF326A9
:106F2800000EF422600EF324D96E020EF420DA6EFD
:106F3800DF501B6E1A501D6E1BC01EF01F50060D31
:106F4800C20EF324136EF00EF420146E1DC015F05B
:106F58001EC016F0000E5EEC4EF01F50060D030E1C
:106F6800F326000EF422600EF324D96E020EF420EC
:106F7800DA6EDF501A6E1F50060D050EF326000E4E
:106F8800F422600EF324D96E020EF420DA6EDF507C
:106F98001B6E1A501D6E1BC01EF01F50060DC40E2E
:106FA800F324136EF00EF420146E1DC015F01EC0ED
:106FB80016F0000E5EEC4EF01F2A070E1F64E7EF76
:106FC80037F0E9EF37F057EF37F0EBEF37F0000E17
:106FD8001F6E070E1F64F3EF37F0F5EF37F0F9EF88
:106FE80037F08DEF38F08DEF38F01F50060D300E6A
:106FF800F324D96E010EF420DA6EDF501A6E1F509A
:10700800060D010EF326000EF422300EF324D96E7D
:10701800010EF420DA6EDF501B6E1A501D6E1BC075
:107028001EF01F50060DF00EF324136EF00EF42020
:10703800146E1DC015F01EC016F0000E5EEC4EF06A
:107048001F50060D020EF326000EF422300EF32414
:10705800D96E010EF420DA6EDF501A6E1F50060D3D
:10706800040EF326000EF422300EF324D96E010E1E
:10707800F420DA6EDF501B6E1A501D6E1BC01EF016
:107088001F50060DF20EF324136EF00EF420146E4A
:107098001DC015F01EC016F0000E5EEC4EF01F501D
:1070A800060D030EF326000EF422300EF324D96EDB
:1070B800010EF420DA6EDF501A6E1F50060D050E11
:1070C800F326000EF422300EF324D96E010EF420BC
:1070D800DA6EDF501B6E1A501D6E1BC01EF01F505B
:1070E800060DF40EF324136EF00EF420146E1DC07A
:1070F80015F01EC016F0000E5EEC4EF01F2A070EAB
:107108001F6489EF38F08BEF38F0F9EF37F08DEF27
:1071180038F0000E1F6E070E1F6495EF38F097EFDA
:1071280038F09BEF38F02FEF39F02FEF39F01F5080
:10713800060D300EF324D96E020EF420DA6EDF50FD
:107148001A6E1F50060D010EF326000EF422300EA3
:10715800F324D96E020EF420DA6EDF501B6E1A503B
:107168001D6E1BC01EF01F50060D200EF324136E5B
:10717800F10EF420146E1DC015F01EC016F0000E9E
:107188005EEC4EF01F50060D020EF326000EF422A0
:10719800300EF324D96E020EF420DA6EDF501A6E28
:1071A8001F50060D040EF326000EF422300EF324B1
:1071B800D96E020EF420DA6EDF501B6E1A501D6E67
:1071C8001BC01EF01F50060D220EF324136EF10E85
:1071D800F420146E1DC015F01EC016F0000E5EECF3
:1071E8004EF01F50060D030EF326000EF422300E4B
:1071F800F324D96E020EF420DA6EDF501A6E1F5097
:10720800060D050EF326000EF422300EF324D96E77
:10721800020EF420DA6EDF501B6E1A501D6E1BC072
:107228001EF01F50060D240EF324136EF10EF420E9
:10723800146E1DC015F01EC016F0000E5EEC4EF068
:107248001F2A070E1F642BEF39F02DEF39F09BEF43
:1072580038F02FEF39F0000E1F6E070E1F6437EF5E
:1072680039F039EF39F03DEF39F0D1EF39F0D1EF9E
:1072780039F01F50060D000EF324D96E020EF420CB
:10728800DA6EDF501A6E1F50060D010EF326000E3F
:10729800F422000EF324D96E020EF420DA6EDF50C9
:1072A8001B6E1A501D6E1BC01EF01F50060D500E8F
:1072B800F324136EF10EF420146E1DC015F01EC0D9
:1072C80016F0000E5EEC4EF01F50060D020EF3266F
:1072D800000EF422000EF324D96E020EF420DA6EAA
:1072E800DF501A6E1F50060D040EF326000EF4220E
:1072F800000EF324D96E020EF420DA6EDF501B6EF6
:107308001A501D6E1BC01EF01F50060D520EF3249E
:10731800136EF10EF420146E1DC015F01EC016F089
:10732800000E5EEC4EF01F50060D030EF326000E05
:10733800F422000EF324D96E020EF420DA6EDF5028
:107348001A6E1F50060D050EF326000EF422000ECD
:10735800F324D96E020EF420DA6EDF501B6E1A5039
:107368001D6E1BC01EF01F50060D540EF324136E25
:10737800F10EF420146E1DC015F01EC016F0000E9C
:107388005EEC4EF01F2A070E1F64CDEF39F0CFEFE9
:1073980039F03DEF39F0D1EF39F00001C0511A6EE4
:1073A800BF511D6E1AC01EF0F10E146E800E136EC2
:1073B8001DC015F01EC016F0000E5EEC4EF0000168
:1073C800C2511A6EC1511D6E1AC01EF0F10E146E14
:1073D800820E136E1DC015F01EC016F0000E5EEC76
:1073E8004EF00001C4511A6EC3511D6E1AC01EF032
:1073F800F10E146E840E136E1DC015F01EC016F02B
:10740800000E5EEC4EF00001C6511A6EC5511D6E9D
:107418001AC01EF0F10E146E860E136E1DC015F004
:107428001EC016F0000E5EEC4EF000018D511A6E73
:107438008C511D6E1AC01EF0F10E146E880E136E5C
:107448001DC015F01EC016F0000E5EEC4EF00001D7
:107458008F511A6E8E511D6E1AC01EF0F10E146EE9
:107468008A0E136E1DC015F01EC016F0000E5EECDD
:107478004EF0000191511A6E90511D6E1AC01EF007
:10748800F10E146E8C0E136E1DC015F01EC016F092
:10749800000E5EEC4EF0000193511A6E92511D6E73
:1074A8001AC01EF0F10E146E8E0E136E1DC015F06C
:1074B8001EC016F0000E5EEC4EF047501A6E485093
:1074C8001D6E1AC01EF0F10E146E900E136E1DC0C4
:1074D80015F01EC016F0000E5EEC4EF045501A6E08
:1074E80046501D6E1AC01EF0F10E146E920E136EE9
:1074F8001DC015F01EC016F0000E5EEC4EF0F10E29
:10750800146E940E136E2AC015F02BC016F0000EE0
:107518005EEC4EF0000E1F6E070E1F6496EF3AF0F9
:1075280098EF3AF09CEF3AF030EF3BF030EF3BF059
:107538001F50060D000EF324D96E010EF420DA6EEA
:10754800DF501A6E1F50060D010EF326000EF422AE
:10755800000EF324D96E010EF420DA6EDF501B6E94
:107568001A501D6E1BC01EF01F50060D960EF324F8
:10757800136EF10EF420146E1DC015F01EC016F027
:10758800000E5EEC4EF01F50060D020EF326000EA4
:10759800F422000EF324D96E010EF420DA6EDF50C7
:1075A8001A6E1F50060D040EF326000EF422000E6C
:1075B800F324D96E010EF420DA6EDF501B6E1A50D8
:1075C8001D6E1BC01EF01F50060D980EF324136E7F
:1075D800F10EF420146E1DC015F01EC016F0000E3A
:1075E8005EEC4EF01F50060D030EF326000EF4223B
:1075F800000EF324D96E010EF420DA6EDF501A6EF5
:107608001F50060D050EF326000EF422000EF3247B
:10761800D96E010EF420DA6EDF501B6E1A501D6E03
:107628001BC01EF01F50060D9A0EF324136EF10EA8
:10763800F420146E1DC015F01EC016F0000E5EEC8E
:107648004EF01F2A070E1F642CEF3BF02EEF3BF085
:107658009CEF3AF030EF3BF0000E1F6E1200BBECCF
:107668004DF0A9C0F9F2AAC0FAF2000E0201FB6FB0
:10767800090EFB6542EF3BF044EF3BF048EF3BF06F
:107688005BEF3BF05BEF3BF0FB51010DEF0EF3249A
:10769800D96E020EF420DA6E2D0EDF6EFB2B090E6A
:1076A800FB6559EF3BF05BEF3BF048EF3BF02CA05C
:1076B80060EF3BF062EF3BF06FEF3BF02DBE67EF02
:1076C8003BF069EF3BF06FEF3BF02C902D8E86EC92
:1076D80041F084EF40F02CA274EF3BF076EF3BF0E2
:1076E800F4EF3BF02DBE7BEF3BF07DEF3BF0F4EF8A
:1076F8003BF02C922D8E000EFB6F070EFB6587EF7B
:107708003BF089EF3BF08DEF3BF084EF40F084EFE6
:1077180040F0FB51060D020EF326000EF422C00EB7
:10772800F324D96E010EF420DA6EF951DE18D8A4CC
:10773800A0EF3BF0A2EF3BF0E6EF3BF0FB51060D6C
:10774800040EF326000EF422C00EF324D96E010EA7
:10775800F420DA6EFA51DE18D8A4B5EF3BF0B7EF93
:107768003BF0E6EF3BF04C0EEF6F310EF06F300E52
:10777800F16F300EF26FFB51060D010EF326000E6D
:10778800F422C00EF324D96E010EF420DA6E590EDD
:10779800DE18D8A4D2EF3BF0D4EF3BF0D8EF3BF0A3
:1077A800310EF36FDCEF3BF0300EF36FDCEF3BF0A4
:1077B800EF0E1B6E020E1C6E0A0E1D6E04EC4BF0D3
:1077C800E6EF3BF00201FB2B070EFB65EEEF3BF00B
:1077D800F0EF3BF08DEF3BF084EF40F084EF40F0AA
:1077E8002CA4F9EF3BF0FBEF3BF079EF3CF02DBE1A
:1077F80000EF3CF002EF3CF079EF3CF02C942D8E3A
:10780800000EFB6F070EFB650CEF3CF00EEF3CF033
:1078180012EF3CF084EF40F084EF40F0FB51060D8E
:10782800020EF326000EF422900EF324D96E010EF8
:10783800F420DA6EF951DE18D8A425EF3CF027EFD2
:107848003CF06BEF3CF0FB51060D040EF326000EE6
:10785800F422900EF324D96E010EF420DA6EFA5158
:10786800DE18D8A43AEF3CF03CEF3CF06BEF3CF06C
:107878004C0EEF6F320EF06F300EF16F300EF26F6C
:10788800FB51060D010EF326000EF422900EF32490
:10789800D96E010EF420DA6E590EDE18D8A457EF0F
:1078A8003CF059EF3CF05DEF3CF0310EF36F61EFC7
:1078B8003CF0300EF36F61EF3CF0EF0E1B6E020EE2
:1078C8001C6E0A0E1D6E04EC4BF06BEF3CF00201CF
:1078D800FB2B070EFB6573EF3CF075EF3CF012EFE6
:1078E8003CF084EF40F084EF40F02CA67EEF3CF0B3
:1078F80080EF3CF0FEEF3CF02DBE85EF3CF087EFCB
:107908003CF0FEEF3CF02C962D8E000EFB6F070E20
:10791800FB6591EF3CF093EF3CF097EF3CF084EF80
:1079280040F084EF40F0FB51060D020EF326000EE6
:10793800F422600EF324D96E010EF420DA6EF951A8
:10794800DE18D8A4AAEF3CF0ACEF3CF0F0EF3CF026
:10795800FB51060D040EF326000EF422600EF324EC
:10796800D96E010EF420DA6EFA51DE18D8A4BFEFF2
:107978003CF0C1EF3CF0F0EF3CF04C0EEF6F330EF3
:10798800F06F300EF16F300EF26FFB51060D010EE5
:10799800F326000EF422600EF324D96E010EF420B3
:1079A800DA6E590EDE18D8A4DCEF3CF0DEEF3CF0BE
:1079B800E2EF3CF0310EF36FE6EF3CF0300EF36F80
:1079C800E6EF3CF0EF0E1B6E020E1C6E0A0E1D6EEB
:1079D80004EC4BF0F0EF3CF00201FB2B070EFB65CB
:1079E800F8EF3CF0FAEF3CF097EF3CF084EF40F012
:1079F80084EF40F02DA003EF3DF005EF3DF07DEF63
:107A08003DF02DBE0AEF3DF00CEF3DF07DEF3DF06F
:107A18002D902D8E000EFB6F070EFB6516EF3DF0C7
:107A280018EF3DF01CEF3DF084EF40F084EF40F09C
:107A3800FB51060D020EF326000EF422900EF324DD
:107A4800D96E020EF420DA6EF951DE18D8A42FEFA1
:107A58003DF031EF3DF06FEF3DF0FB51060D040EA8
:107A6800F326000EF422900EF324D96E020EF420B1
:107A7800DA6EFA51DE18D8A444EF3DF046EF3DF037
:107A88006FEF3DF0460EEF6FFB51060D010EF3262A
:107A9800000EF422900EF324D96E020EF420DA6E52
:107AA800590EDE18D8A45BEF3DF05DEF3DF061EFB5
:107AB8003DF0310EF06F65EF3DF0300EF06F65EF81
:107AC8003DF0EF0E1B6E020E1C6E0A0E1D6E04ECCE
:107AD8004BF06FEF3DF00201FB2B070EFB6577EFD4
:107AE8003DF079EF3DF01CEF3DF084EF40F084EF7E
:107AF80040F02CAE82EF3DF084EF3DF0FCEF3DF01E
:107B08002DBE89EF3DF08BEF3DF0FCEF3DF02C9E54
:107B18002D8E000EFB6F070EFB6595EF3DF097EF7E
:107B28003DF09BEF3DF084EF40F084EF40F0FB51D7
:107B3800060D020EF326000EF422600EF324D96E11
:107B4800020EF420DA6EF951DE18D8A4AEEF3DF03B
:107B5800B0EF3DF0EEEF3DF0FB51060D040EF326BD
:107B6800000EF422600EF324D96E020EF420DA6EB1
:107B7800FA51DE18D8A4C3EF3DF0C5EF3DF0EEEFA3
:107B88003DF0530EEF6FFB51060D010EF326000E6C
:107B9800F422600EF324D96E020EF420DA6E590E28
:107BA800DE18D8A4DAEF3DF0DCEF3DF0E0EF3DF071
:107BB800310EF06FE4EF3DF0300EF06FE4EF3DF082
:107BC800EF0E1B6E020E1C6E0A0E1D6E04EC4BF0BF
:107BD800EEEF3DF00201FB2B070EFB65F6EF3DF0E3
:107BE800F8EF3DF09BEF3DF084EF40F084EF40F07C
:107BF8002CA801EF3EF003EF3EF081EF3EF02DBEE2
:107C080008EF3EF00AEF3EF081EF3EF02C982D8E03
:107C1800000EFB6F070EFB6514EF3EF016EF3EF00B
:107C28001AEF3EF084EF40F084EF40F0FB51060D70
:107C3800020EF326000EF422300EF324D96E010E44
:107C4800F420DA6EF951DE18D8A42DEF3EF02FEFAC
:107C58003EF073EF3EF0FB51060D040EF326000EC6
:107C6800F422300EF324D96E010EF420DA6EFA51A4
:107C7800DE18D8A442EF3EF044EF3EF073EF3EF03A
:107C8800430EEF6F310EF06F300EF16F300EF26F62
:107C9800FB51060D010EF326000EF422300EF324DC
:107CA800D96E010EF420DA6E590EDE18D8A45FEFF3
:107CB8003EF061EF3EF065EF3EF0310EF36F69EF95
:107CC8003EF0300EF36F69EF3EF0EF0E1B6E020EC2
:107CD8001C6E0A0E1D6E04EC4BF073EF3EF00201B1
:107CE800FB2B070EFB657BEF3EF07DEF3EF01AEFB6
:107CF8003EF084EF40F084EF40F02CAA86EF3EF08F
:107D080088EF3EF006EF3FF02DBE8DEF3EF08FEF8F
:107D18003EF006EF3FF02C9A2D8E000EFB6F070EFB
:107D2800FB6599EF3EF09BEF3EF09FEF3EF084EF4E
:107D380040F084EF40F0FB51060D020EF326000ED2
:107D4800F422300EF324D96E020EF420DA6EF951C3
:107D5800DE18D8A4B2EF3EF0B4EF3EF0F8EF3EF0F4
:107D6800FB51060D040EF326000EF422300EF32408
:107D7800D96E020EF420DA6EFA51DE18D8A4C7EFD5
:107D88003EF0C9EF3EF0F8EF3EF0430EEF6F320ED3
:107D9800F06F300EF16F300EF26FFB51060D010ED1
:107DA800F326000EF422300EF324D96E020EF420CE
:107DB800DA6E590EDE18D8A4E4EF3EF0E6EF3EF096
:107DC800EAEF3EF0310EF36FEEEF3EF0300EF36F58
:107DD800EEEF3EF0EF0E1B6E020E1C6E0A0E1D6ECD
:107DE80004EC4BF0F8EF3EF00201FB2B070EFB65AD
:107DF80000EF3FF002EF3FF09FEF3EF084EF40F0DE
:107E080084EF40F02CAC0BEF3FF00DEF3FF08BEF21
:107E18003FF02DBE12EF3FF014EF3FF08BEF3FF035
:107E28002C9C2D8E000EFB6F070EFB651EEF3FF09E
:107E380020EF3FF024EF3FF084EF40F084EF40F074
:107E4800FB51060D020EF326000EF422000EF32459
:107E5800D96E020EF420DA6EF951DE18D8A437EF85
:107E68003FF039EF3FF07DEF3FF0FB51060D040E78
:107E7800F326000EF422000EF324D96E020EF4202D
:107E8800DA6EFA51DE18D8A44CEF3FF04EEF3FF00F
:107E98007DEF3FF0430EEF6F330EF06F300EF16F52
:107EA800300EF26FFB51060D010EF326000EF42280
:107EB800000EF324D96E020EF420DA6E590EDE1885
:107EC800D8A469EF3FF06BEF3FF06FEF3FF0310E52
:107ED800F36F73EF3FF0300EF36F73EF3FF0EF0E79
:107EE8001B6E020E1C6E0A0E1D6E04EC4BF07DEF2D
:107EF8003FF00201FB2B070EFB6585EF3FF087EF94
:107F08003FF024EF3FF084EF40F084EF40F02DA2E3
:107F180090EF3FF092EF3FF09DEF3FF02DBE97EFCF
:107F28003FF099EF3FF09DEF3FF02D922D8E84EFBB
:107F380040F02DA4A2EF3FF0A4EF3FF0AFEF3FF0E9
:107F48002DBEA9EF3FF0ABEF3FF0AFEF3FF02D9420
:107F58002D8E84EF40F02DA6B4EF3FF0B6EF3FF042
:107F6800C1EF3FF02DBEBBEF3FF0BDEF3FF0C1EFDB
:107F78003FF02D962D8E84EF40F02DA8C6EF3FF0F0
:107F8800C8EF3FF0D3EF3FF02DBECDEF3FF0CFEF7E
:107F98003FF0D3EF3FF02D982D8E84EF40F02DAABF
:107FA800D8EF3FF0DAEF3FF084EF40F02DBEDFEF7F
:107FB8003FF0E1EF3FF084EF40F02D9A2D8E000E58
:107FC800FB6F070EFB65EBEF3FF0EDEF3FF0F1EFD6
:107FD8003FF084EF40F084EF40F0FB51060D020EB5
:107FE800F326000EF422000EF324D96E010EF420BD
:107FF800DA6EF951DE18D8A404EF40F006EF40F02D
:108008005EEF40F0FB51060D040EF326000EF4223D
:10801800000EF324D96E010EF420DA6EFA51DE1840
:10802800D8A419EF40F01BEF40F05EEF40F0520E7D
:10803800EF6F310EF06FFB51060D000EF324D96E71
:10804800010EF420DA6EDF50F16FFB51060D050EBC
:10805800F326000EF422000EF324D96E010EF4204C
:10806800DA6EDF50F26FFB51060D010EF326000E9B
:10807800F422000EF324D96E010EF420DA6E590EA4
:10808800DE18D8A44AEF40F04CEF40F050EF40F033
:10809800310EF36F54EF40F0300EF36F54EF40F0B1
:1080A800EF0E1B6E020E1C6E0A0E1D6E04EC4BF0DA
:1080B8005EEF40F00201FB2B070EFB6566EF40F018
:1080C80068EF40F0F1EF3FF084EF40F084EF40F0CC
:1080D80084EF40F084EF40F084EF40F084EF40F00C
:1080E80084EF40F084EF40F084EF40F084EF40F0FC
:1080F80084EF40F084EF40F084EF40F084EF40F0EC
:108108002D9EFF0E206E3F0E216E2CC022F02DC03A
:1081180023F0205022162150231622502310D8A4D1
:1081280098EF40F09AEF40F0A0EF40F0FF0E2C12CD
:108138003F0E2D12A0EF40F01200176E080E156EBC
:108148000B0EF7EC4FF0000E156E0C0EF7EC4FF01F
:10815800E5EF40F0210E156E0D0EF7EC4FF0620EB4
:10816800156E0E0EF7EC4FF0760E156E0F0EF7EC3F
:108178004FF0F4EF40F0220E156E0D0EF7EC4FF0B5
:10818800B10E156E0E0EF7EC4FF03B0E156E0F0E7E
:10819800F7EC4FF0F4EF40F0100E156E0D0EF7EC03
:1081A8004FF0A70E156E0E0EF7EC4FF0620E156E1F
:1081B8000F0EF7EC4FF0F4EF40F0F4EF40F0F4EF6F
:1081C80040F01750000AD8B4BFEF40F0010AD8B405
:1081D800D0EF40F0030AD8B4AEEF40F0F4EF40F02F
:1081E8005B0E156E100EF7EC4FF0F80E156E110EB3
:1081F800F7EC4FF0030E156E120EF7EC4FF0220E4F
:10820800156E130EF7EC4FF0F80E156E140EF7EC12
:108218004FF0000E156E0A0EF7EC4FF0470E156E74
:10822800150EF7EC4FF0B60E156E210EF7EC4FF069
:10823800100E156E220EF7EC4FF0190E156E180E73
:10824800F7EC4FF01D0E156E190EF7EC4FF01C0EE3
:10825800156E1A0EF7EC4FF0C70E156E1B0EF7ECE5
:108268004FF0000E156E1C0EF7EC4FF0B20E156EA7
:108278001D0EF7EC4FF0EA0E156E230EF7EC4FF0DB
:108288002A0E156E240EF7EC4FF0000E156E250E13
:10829800F7EC4FF0110E156E260EF7EC4FF0590E55
:1082A800156E290EF7EC4FF0810E156E2C0EF7ECBB
:1082B8004FF0350E156E2D0EF7EC4FF0090E156EBA
:1082C8002E0EF7EC4FF00B0E156E000EF7EC4FF07C
:1082D800060E156E020EF7EC4FF0040E156E070E23
:1082E800F7EC4FF0050E156E080EF7EC4FF0000E88
:1082F800156E090EF7EC4FF03D0E156E060EF7ECF5
:108308004FF01200BBEC4DF0540E0401826F200EAA
:10831800836F5B0E846FA6C013F0146A000E166E8E
:108328000A0E156E7BEC45F01350300F0401856F73
:10833800A6C013F0146A000E166E0A0E156E61ECD4
:1083480046F01350300F0401866F2F0E876FA7C0B9
:1083580013F0146A000E166E0A0E156E7BEC45F0CB
:108368001350300F0401886FA7C013F0146A000E71
:10837800166E0A0E156E61EC46F01350300F0401AC
:10838800896F2F0E8A6FA8C013F0146A000E166E3C
:108398000A0E156E7BEC45F01350300F04018B6FFD
:1083A800A8C013F0146A000E166E0A0E156E61EC62
:1083B80046F01350300F04018C6F200E8D6FA9C04A
:1083C80013F0146A000E166E0A0E156E7BEC45F05B
:1083D8001350300F04018E6FA9C013F0146A000EF9
:1083E800166E0A0E156E61EC46F01350300F04013C
:1083F8008F6F3A0E906FAAC013F0146A000E166EB3
:108408000A0E156E7BEC45F01350300F0401916F86
:10841800AAC013F0146A000E166E0A0E156E61ECEF
:1084280046F01350300F0401926F3A0E936FABC0B1
:1084380013F0146A000E166E0A0E156E7BEC45F0EA
:108448001350300F0401946FABC013F0146A000E80
:10845800166E0A0E156E61EC46F01350300F0401CB
:10846800956F5D0E966F0A0E976F820E1B6E040E47
:108478001C6E150E1D6E04EC4BF01200F7C221F0B5
:10848800226A236A0201F635213601E3228021504F
:10849800FE6FFE51D8A453EF42F055EF42F061EF62
:1084A80042F0000EF56F000EF66F000EF76F000E2B
:1084B800F86FF8EF42F0F8EF42F0170E216EF5C2B0
:1084C80022F0F6C223F0F7C224F02128256E71EFBE
:1084D80042F0D890243223322232252E6DEF42F01A
:1084E80022500201F96FF68FFF0EF517FF0EF617EF
:1084F800000EF717F551FA6FF651FB6FF751FC6F45
:10850800FD6B8E0EFE5FFEBF8EEF42F08CEF42F0E9
:10851800B2EF42F0FE51800A8F0FD8B096EF42F0CA
:1085280098EF42F0A6EF42F0000EF56F000EF66FDE
:10853800000EF76F000EF86FF8EF42F0F8EF42F018
:10854800A6EF42F0D890FD33FC33FB33FA33FE3FFD
:10855800A6EF42F0DCEF42F0DCEF42F0170EFE65CA
:10856800B8EF42F0BAEF42F0D0EF42F0000EF56FEC
:10857800000EF66F000EF76F000EF86FF8EF42F07E
:10858800F8EF42F0D0EF42F0D890FA37FB37FC37DB
:10859800FD37FE07D0EF42F0FE51D8A4D6EF42F0E7
:1085A800D8EF42F0C8EF42F0DCEF42F0DCEF42F0E7
:1085B800F951D8B4E2EF42F0E4EF42F0EEEF42F0C6
:1085C800FD1FFC1FFB1FFA6D000EFB23FC23FD2380
:1085D800EEEF42F0FAC2F5F2FBC2F6F2FCC2F7F295
:1085E800FDC2F8F2F8EF42F01200FACF01F0FBCF2B
:1085F80002F0E9CF03F0EACF04F0E1CF05F0E2CFD3
:1086080006F0D9CF07F0DACF08F0F3CF09F0F4CFAE
:108618000AF0F6CF0BF0F7CF0CF0F8CF0DF0F5CF4E
:108628000EF04DC00FF04EC010F04FC011F050C00A
:1086380012F0F2AA22EF43F024EF43F034EF43F0B4
:10864800F2A429EF43F02BEF43F034EF43F0B10EDF
:10865800D76EE00ED66E010E436EF29488EF43F0AB
:108668009DA839EF43F03BEF43F047EF43F09EA856
:1086780040EF43F042EF43F047EF43F012EC4EF087
:108688009E9888EF43F09DAA4CEF43F04EEF43F0DD
:108698005AEF43F09EAA53EF43F055EF43F05AEFD9
:1086A80043F083EC4EF09E9A88EF43F0A3A85FEF67
:1086B80043F061EF43F06DEF43F0A4A866EF43F099
:1086C80068EF43F06DEF43F038EC4EF0A49888EF74
:1086D80043F0A3AA72EF43F074EF43F088EF43F03E
:1086E800A4AA79EF43F07BEF43F088EF43F0A7ECBF
:1086F8004EF0A49A88EF43F088EF43F088EF43F0F8
:1087080088EF43F088EF43F012C050F011C04FF0EB
:1087180010C04EF00FC04DF00EC0F5FF0DC0F8FFB1
:108728000CC0F7FF0BC0F6FF0AC0F4FF09C0F3FF47
:1087380008C0DAFF07C0D9FF06C0E2FF05C0E1FFA5
:1087480004C0EAFF03C0E9FF02C0FBFF01C0FAFF53
:108758004D921100DEC01EF01F6A206A0001DD354F
:108768001E3601E31F801E500201F36FF351D8A497
:10877800C0EF43F0C2EF43F0CDEF43F0000E00012D
:10878800DC6F000EDD6F000EDE6F4BEF44F04BEF39
:1087980044F0E1C01EF01F6A206A0001E0351E3671
:1087A80001E31F801E500201F46FF451D8A4DFEFDB
:1087B80043F0E1EF43F0ECEF43F0000E0001DC6F13
:1087C800000EDD6F000EDE6F4BEF44F04BEF44F010
:1087D800000E0201F06F000EF16F000EF26FF451FF
:1087E800890FF35FDEC0F4F20001E1510201F41BCE
:1087F800800EF4170001DD8FFF0EDC17FF0EDD176A
:10880800000EDE17E08FFF0EDF17FF0EE017000ED9
:10881800E117180E0201EF6F12EF44F0D890F0370D
:10882800F137F2370001DF51DC5DE051DD59E151EC
:10883800DE59D8A022EF44F024EF44F02CEF44F0A6
:10884800DF51DC5FE051DD5BE151DE5B0201F0816D
:108858000001D890DC37DD37DE370201EF2F12EF49
:1088680044F037EF44F0F0C213F0F1C214F0F2C252
:1088780015F0F3C216F0F4C217F04CEC44F013C034
:10888800DCF014C0DDF015C0DEF04BEF44F0120050
:108898001650D8B452EF44F054EF44F060EF44F06F
:1088A800135014101510D8A45CEF44F05EEF44F098
:1088B80073EF44F060EF44F0000E136E000E146E78
:1088C800000E156EE7EF44F0E7EF44F073EF44F065
:1088D800162AD89015321432133273EF44F0000E72
:1088E8001314186E000E1414196EFE0E15141A6E59
:1088F800185019101A10D8A484EF44F086EF44F0E9
:108908006CEF44F097EF44F097EF44F0162A010E0D
:108918001326000E1422000E1522D8901532143298
:10892800133297EF44F0000E1314186E000E14144F
:10893800196EFF0E15141A6E185019101A10D8A4B3
:10894800A8EF44F0AAEF44F08AEF44F0B5EF44F002
:10895800B5EF44F01606D890133614361536B5EF31
:1089680044F014BEBAEF44F0BCEF44F0C6EF44F054
:10897800020E1660C2EF44F0C4EF44F0AEEF44F0CC
:10898800C6EF44F016B0CBEF44F0CDEF44F0D0EF93
:1089980044F0149ED0EF44F0D890163216501512B9
:1089A8001750D8B4DAEF44F0DCEF44F0DFEF44F0CE
:1089B800158EDFEF44F013C013F014C014F015C087
:1089C80015F0E7EF44F012001AC013F01BC014F0C2
:1089D800000E166E0A0E156E55EC4AF013C024F000
:1089E80014C025F01AC013F01BC014F0000E166E48
:1089F8000A0E156E4FEC49F013C01AF014C01BF0A4
:108A08001AC013F01BC014F0000E166E0A0E156E75
:108A180055EC4AF013C022F014C023F01AC013F02A
:108A28001BC014F0000E166E0A0E156E4FEC49F0BE
:108A380013C01AF014C01BF01AC013F01BC014F0B6
:108A4800000E166E0A0E156E55EC4AF013C020F093
:108A580014C021F01AC013F01BC014F0000E166EDB
:108A68000A0E156E4FEC49F013C01AF014C01BF033
:108A78001AC013F01BC014F0000E166E0A0E156E05
:108A880055EC4AF013C01EF014C01FF01AC013F0C2
:108A98001BC014F0000E166E0A0E156E4FEC49F04E
:108AA80013C01AF014C01BF01AC013F01BC014F046
:108AB800000E166E0A0E156E55EC4AF013C01CF027
:108AC80014C01DF01C50300FDCEC4BF01E50300F62
:108AD800DCEC4BF02050300FDCEC4BF02250300F28
:108AE800DCEC4BF02450300FDCEC4BF01200000EA5
:108AF800186E16BE84EF45F082EF45F08CEF45F016
:108B0800156C161ED8B0162A010E186E8CEF45F09B
:108B180014BE93EF45F091EF45F09BEF45F0136CD1
:108B2800141ED8B0142A010E181A9BEF45F0000E37
:108B38001A6E000E196E15501610D8B4A6EF45F02F
:108B4800A8EF45F0DCEF45F0010E176EB2EF45F0E7
:108B5800D89015361636172AB2EF45F016AEB7EF8D
:108B680045F0B9EF45F0ACEF45F0BDEF45F0BDEF8E
:108B780045F0D89019361A361550135C165014580B
:108B8800D8A0C9EF45F0CBEF45F0D2EF45F015502E
:108B9800135E1650145A1980D2EF45F0D890163249
:108BA8001532172EBDEF45F0DCEF45F0DCEF45F050
:108BB8001850D8B4E2EF45F0E4EF45F0EAEF45F09D
:108BC800196C1A1ED8B01A2AEAEF45F019C013F02A
:108BD8001AC014F0F0EF45F01200000E156E640E86
:108BE800146E3B50D8A4FBEF45F0FDEF45F060EF65
:108BF80046F0000E136E070E136405EF46F007EFFC
:108C080046F00BEF46F060EF46F060EF46F00C0ED2
:108C1800BA6E000E156E000E146EF40E145C010E82
:108C28001558D8A01AEF46F01CEF46F020EF46F092
:108C38002FEF46F02FEF46F0144A152AF40E145C75
:108C4800010E1558D8A02BEF46F02DEF46F020EF77
:108C580046F02FEF46F0000EBA6E000E156E000EAD
:108C6800146EE80E145C030E1558D8A03EEF46F0BB
:108C780040EF46F044EF46F053EF46F053EF46F02E
:108C8800144A152AE80E145C030E1558D8A04FEFA5
:108C980046F051EF46F044EF46F053EF46F0132A02
:108CA800070E13645AEF46F05CEF46F00BEF46F000
:108CB80060EF46F060EF46F01200000E186E14BE2A
:108CC8006AEF46F068EF46F072EF46F0136C141E38
:108CD800D8B0142A010E186E72EF46F016BE79EF5E
:108CE80046F077EF46F07FEF46F0156C161ED8B0C9
:108CF800162A7FEF46F015501610D8B486EF46F0C6
:108D080088EF46F0B8EF46F0010E176E92EF46F086
:108D1800D89015361636172A92EF46F016AE97EF0A
:108D280046F099EF46F08CEF46F09DEF46F09DEF48
:108D380046F01550135C16501458D8A0A6EF46F00C
:108D4800A8EF46F0AEEF46F01550135E1650145AD1
:108D5800AEEF46F0D89016321532172E9DEF46F03A
:108D6800B8EF46F0B8EF46F01850D8B4BEEF46F06A
:108D7800C0EF46F0C6EF46F0136C141ED8B0142AA4
:108D8800C6EF46F013C013F014C014F0CCEF46F051
:108D980012003BEC4BF0EBEC4EF04B0E146EEB0E6E
:108DA800156E010E166EE7EC4DF02DEC2EF0DDEF92
:108DB80046F0AEEC48F00001BE05D8A4E6EF46F058
:108DC800E8EF46F0ECEF46F0000EBE6FECEF46F031
:108DD800BD05D8A4F2EF46F0F4EF46F013EF47F0E4
:108DE80078EC00F0FDEC47F089BCFDEF46F000EFB1
:108DF80047F0010E01EF47F0000E00080201FF6F77
:108E0800010EFF27FF3BFF47FF478950FF19BF0BA4
:108E1800FF19896E000E0001BD6F13EF47F0BC0506
:108E2800D8A419EF47F01BEF47F024EF47F04EECBA
:108E380018F033EC3BF0000E0001BC6F24EF47F054
:108E4800BB05D8A42AEF47F02CEF47F0DDEF46F03A
:108E5800010EB96F000EBB6FDDEF46F0DDEF46F097
:108E6800DDEF46F076EF00F000019751D00F176E56
:108E78001750060DF3501324D96EF4501420DA6EEF
:108E880094C0DFFF1750060D13C015F014C016F07C
:108E9800F3501526F4501622010E1524D96E000E33
:108EA8001620DA6E95C0DFFF1750060D13C015F0B7
:108EB80014C016F0F3501526F4501622020E15248D
:108EC800D96E000E1620DA6E96C0DFFF1750060D19
:108ED80013C015F014C016F0F3501526F4501622DE
:108EE800030E1524D96E000E1620DA6E97C0DFFF28
:108EF8001750060D13C015F014C016F0F3501526C0
:108F0800F4501622040E1524D96E000E1620DA6EBF
:108F180098C0DFFF1750060D13C015F014C016F0E7
:108F2800F3501526F4501622050E1524D96E000E9E
:108F38001620DA6E99C0DFFF1200000E1B6E000EBD
:108F48001C6E000E1D6E000E1E6E175018101910A4
:108F58001A10D8B4B2EF47F0B4EF47F0F4EF47F087
:108F6800010E1F6EC0EF47F0D89017361836193625
:108F78001A361F2AC0EF47F01AAEC5EF47F0C7EF01
:108F880047F0B8EF47F0CBEF47F0CBEF47F0D8907A
:108F98001B361C361D361E361750135C18501458D5
:108FA800195015581A501658D8A0DDEF47F0DFEFC2
:108FB80047F0EAEF47F01750135E1850145A19504B
:108FC800155A1A50165A1B80EAEF47F0D8901A32F1
:108FD8001932183217321F2ECBEF47F0F4EF47F053
:108FE8001BC013F01CC014F01DC015F01EC016F0F5
:108FF80012004B04D8A403EF48F005EF48F058EFEF
:1090080048F00A0E4C18D8A40CEF48F00EEF48F0C0
:109018001EEF48F0C450146EC3500001B46F14C062
:10902800B5F0040E4C6E040E08EC51F038EC51F01B
:1090380054EF48F0040E4C18D8A425EF48F027EF59
:1090480048F037EF48F0C450146EC3500001B26FB7
:1090580014C0B3F00C0E4C6E0C0E08EC51F038EC4A
:1090680051F054EF48F00C0E4C18D8A43EEF48F0DD
:1090780040EF48F054EF48F0C450146EC35000015C
:10908800AE6F14C0AFF00A0E4C6E0A0E08EC51F029
:1090980038EC51F054EF48F054EF48F054EF48F0F2
:1090A800000E4B6E58EF48F01200000EF66EA20E3E
:1090B800F76E000EF86E01EEF0F010EE10F00900F9
:1090C800F5CFEEFFE550E150FAE1440EF66EA20E40
:1090D800F76E000EF86E00EEE3F010EE08F00900EF
:1090E800F5CFEEFFE550E150FAE105EE00F011EEA4
:1090F80000F0EE6AE550E150FCE1E250FAE104EEDE
:1091080000F0820EEE6AE806FDE103EE00F0F40ED0
:10911800EE6AE806FDE102EE00F0EF0EEE6AE80600
:10912800FDE101EE00F0F00EEE6AE806FDE100EE6A
:1091380060F0670EEE6AE806FDE100EE26F0230E09
:10914800EE6AE806FDE14D904D92000EF86E0001C2
:10915800CDEF46F04304D8A4B4EF48F0B6EF48F09A
:1091680000EF49F0010E0001BE6F335007E10A0E0F
:10917800325CD8B0C2EF48F0C4EF48F0C8EF48F00E
:10918800324A332AD0EF48F0000E336E000E326EAA
:10919800010EBD6FD0EF48F0315007E1640E305C2E
:1091A800D8B0D9EF48F0DBEF48F0DFEF48F0304AAD
:1091B800312AE7EF48F0000E316E000E306E010ED6
:1091C800BC6FE7EF48F0E80E2E5C030E2F58D8B0BE
:1091D800F0EF48F0F2EF48F0F6EF48F02E4A2F2A69
:1091E800FCEF48F0000E2F6E000E2E6E010EBB6FC6
:1091F800000E436E00EF49F01200175018101910B6
:109208001A10D8B40AEF49F00CEF49F046EF49F0CC
:10921800010E1B6E18EF49F0D8901736183619361C
:109228001A361B2A18EF49F01AAE1DEF49F01FEF46
:1092380049F010EF49F023EF49F023EF49F01750B8
:10924800135C18501458195015581A501658D8A0AD
:1092580030EF49F032EF49F03CEF49F01750135E18
:109268001850145A1950155A1A50165A3CEF49F00A
:10927800D8901A321932183217321B2E23EF49F0C0
:1092880046EF49F013C013F014C014F015C015F0E0
:1092980016C016F01200000E196E000E186E15504A
:1092A8001610D8B45AEF49F05CEF49F08EEF49F048
:1092B800010E176E66EF49F0D89015361636172A44
:1092C80066EF49F016AE6BEF49F06DEF49F060EFCD
:1092D80049F071EF49F071EF49F0D8901836193616
:1092E8001550135C16501458D8A07DEF49F07FEF45
:1092F80049F086EF49F01550135E1650145A18803D
:1093080086EF49F0D89016321532172E71EF49F0D2
:109318008EEF49F018C013F019C014F012008984B8
:109328008D828D94340E146EEC0E156E000E166E32
:10933800E7EC4DF04AEC26F0C70E146EEF0E156EF2
:10934800010E166EE7EC4DF01F0E146EEC0E156E46
:10935800000E166EE7EC4DF0010EA1EC40F0C70EC2
:10936800146EEF0E156E010E166EE7EC4DF0480EFA
:10937800146EEC0E156E000E166EE7EC4DF0E30E53
:10938800156E000E166E080E176E3E0E73EC4CF03E
:10939800C70E146EEF0E156E010E166EE7EC4DF04B
:1093A8001200176E17380F0B0F0B166E17500F0B96
:1093B800156E300EDCEC4BF0780EDCEC4BF01650F2
:1093C800010DF00EF324D96E010EF420DA6EDF5091
:1093D800DCEC4BF01550010DF00EF324D96E010EA4
:1093E800F420DA6EDF50DCEC4BF01404D8A4FFEF65
:1093F80049F001EF4AF005EF4AF010EC51F015EF93
:109408004AF0020E1418D8A40CEF4AF00EEF4AF0F6
:1094180015EF4AF0200EDCEC4BF015EF4AF015EF93
:109428004AF0120020EE04F01350D9261450DA2224
:1094380088C0DFFF20EE05F01350D9261450DA2239
:1094480089C0DFFF20EE02F01350D9261450DA222B
:1094580086C0DFFF20EE03F01350D9261450DA221D
:1094680087C0DFFF13C0D9FF14C0DAFF84C0DFFF55
:1094780020EE01F01350D9261450DA2285C0DFFF00
:1094880020EE06F01350D9261450DA228AC0DFFFE6
:1094980020EE07F01350D9261450DA228BC0DFFFD4
:1094A800120015501610D8B45CEF4AF05EEF4AF07F
:1094B8008CEF4AF0010E176E68EF4AF0D890153617
:1094C8001636172A68EF4AF016AE6DEF4AF06FEFBE
:1094D8004AF062EF4AF073EF4AF073EF4AF0155022
:1094E800135C16501458D8A07CEF4AF07EEF4AF06F
:1094F80084EF4AF01550135E1650145A84EF4AF060
:10950800D89016321532172E73EF4AF08CEF4AF0C6
:1095180013C013F014C014F01200000E1A6E000EDF
:10952800196E000E186E000E1A6E0F0E1A649FEF59
:109538004AF0A1EF4AF0A5EF4AF0C6EF4AF0C6EFAD
:109548004AF084B0AAEF4AF0AEEF4AF0156A152A3D
:10955800AFEF4AF0156A155018C016F019C017F089
:10956800D890163617361610186E1750196E8D8249
:109578008D921A2A0F0E1A64C4EF4AF0C6EF4AF009
:10958800A5EF4AF018C013F019C014F01200000E2D
:109598001B6E000E1C6E000E1D6E000E1E6ED5EFAB
:1095A8004AF013A0DAEF4AF0DCEF4AF0E6EF4AF0AF
:1095B80017501B2618501C2219501D221A501E2203
:1095C800E6EF4AF0D8901736183619361A36D8907A
:1095D8001632153214321332135014101510161097
:1095E800D8A4F9EF4AF0FBEF4AF0D5EF4AF01BC0D8
:1095F80013F01CC014F01DC015F01EC016F01200A8
:109608001DC015F03F0EF7EC4FF01BC015F01CC045
:1096180016F01DC017F03F0E73EC4CF0350E32EC0F
:1096280050F0000E1F6E000E1E6EE80E1E5C030E3C
:109638001F58D8A022EF4BF024EF4BF028EF4BF047
:1096480037EF4BF037EF4BF01E4A1F2AE80E1E5C2F
:10965800030E1F58D8A033EF4BF035EF4BF028EF2F
:109668004BF037EF4BF03B0E32EC50F01200D38842
:10967800D38AD38CFC0ED31695869594CBEC4FF0F9
:10968800958E95829580EAEC50F09382928A938029
:109698009286E1EC4FF0929CD0EC50F0929E96802E
:1096A80096949692898E8D848D823AEC51F0948EA0
:1096B800949C95988C9844EC50F0939A8A9A76ECFE
:1096C80050F09294928292808984000ED26E000E9D
:1096D800D16ED08EF28EF28C1200216E21502AECBF
:1096E8004FF01F6E090E55EC50F00001DC512AECCA
:1096F8004FF01F6E080E55EC50F00001DD512AECBA
:109708004FF01F6E060E55EC50F00001DE512AECAA
:109718004FF01F6E050E55EC50F00001DF512AEC9A
:109728004FF01F6E040E55EC50F00001E0512AEC8A
:109738004FF01F6E030E55EC50F0000E1F6E020E18
:1097480055EC50F01200136EACEF4BF0ACEF4BF051
:109758004A50D8B4B2EF4BF0B4EF4BF0ACEF4BF04B
:109768009DB8B9EF4BF0BBEF4BF0BFEF4BF013C018
:10977800AEFFDAEF4BF09D984050010D780EF324C0
:10978800D96E000EF420DA6E13C0DFFF402A0B0EEC
:109798004064D1EF4BF0D3EF4BF0D7EF4BF0000E16
:1097A800406ED7EF4BF04A06DAEF4BF09D88120077
:1097B800136EE1EF4BF0E1EF4BF04950D8B4E7EF0F
:1097C8004BF0E9EF4BF0E1EF4BF0A3B8EEEF4BF0C5
:1097D800F0EF4BF0F4EF4BF013C0A9FF0FEF4CF094
:1097E800A3983A50010D400EF324D96E030EF420CD
:1097F800DA6E13C0DFFF3A2A3F0E3A6406EF4CF0E8
:1098080008EF4CF00CEF4CF0000E3A6E0CEF4CF0F9
:1098180049060FEF4CF0A3881200000E156E000EDB
:10982800146E000E156E070E15641DEF4CF01FEF39
:109838004CF023EF4CF03EEF4CF03EEF4CF084B090
:1098480028EF4CF02CEF4CF0136A132A2DEF4CF054
:10985800136A145014241310146E8D828D92152AD5
:10986800070E15643AEF4CF03CEF4CF023EF4CF048
:109878003EEF4CF0145041EF4CF01200000E156E04
:10988800000E146E000E156E070E15644EEF4CF0A8
:1098980050EF4CF054EF4CF06FEF4CF06FEF4CF092
:1098A80084B059EF4CF05DEF4CF0136A132A5EEF69
:1098B8004CF0136A145014241310146E8D828D9278
:1098C800152A070E15646BEF4CF06DEF4CF054EF52
:1098D8004CF06FEF4CF0145072EF4CF01200186E11
:1098E80018504009196E89947AEF4CF084B07FEFD4
:1098F8004CF081EF4CF07AEF4CF083EF4CF01950BC
:1099080031EC4DF0000E1A6E98EF4CF01A50010D24
:10991800F3501524D96EF4501620DA6EDF5031EC6E
:109928004DF01A2A98EF4CF017501A5CD8A09FEF08
:109938004CF0A1EF4CF08AEF4CF089841200196EBC
:109948001950C0091A6E8994AAEF4CF084B0AFEF91
:109958004CF0B1EF4CF0AAEF4CF0B3EF4CF01A50CA
:1099680031EC4DF0000E1B6EC8EF4CF01B50010D92
:10997800F3501624D96EF4501720DA6E11EC4CF01F
:10998800DF6E1B2AC8EF4CF018501B5CD8A0CFEF35
:109998004CF0D1EF4CF0BAEF4CF089841200000E75
:1099A800446EE5EF4CF0442A0A0E4418D8A4DFEFC1
:1099B8004CF0E1EF4CF0E5EF4CF0EEEF4CF0EEEF51
:1099C8004CF073B4EAEF4CF0ECEF4CF0D7EF4CF0FE
:1099D800EEEF4CF00A0E4418D8A4F5EF4CF0F7EF70
:1099E8004CF0FCEF4CF0FF0E02EF4DF002EF4DF0A3
:1099F800718665EC4FF0755002EF4DF01200000EC5
:109A0800136E09EF4DF009EF4DF03C50D8B40FEF4D
:109A18004DF011EF4DF009EF4DF013EF4DF03D50C3
:109A2800010D6C0EF324D96E000EF420DA6EDF50AF
:109A3800136E3D2A0B0E3D6424EF4DF026EF4DF0DA
:109A48002AEF4DF0000E3D6E2AEF4DF09D9A3C0630
:109A58009D8A135030EF4DF01200136E000E146EF5
:109A6800000E146E070E14643CEF4DF03EEF4DF0FF
:109A780042EF4DF05DEF4DF05DEF4DF013AE47EF67
:109A88004DF049EF4DF04CEF4DF08D844FEF4DF018
:109A98008D944FEF4DF013501324136E8D828D92D9
:109AA800142A070E14645BEF4DF05DEF4DF042EFA2
:109AB8004DF08D941200136E000E146E000E146E8D
:109AC800070E14646AEF4DF06CEF4DF070EF4DF037
:109AD8008BEF4DF08BEF4DF013AE75EF4DF077EF48
:109AE8004DF07AEF4DF08D847DEF4DF08D947DEF44
:109AF8004DF013501324136E8D828D92142A070E85
:109B0800146489EF4DF08BEF4DF070EF4DF08D94AC
:109B18001200000E136E93EF4DF093EF4DF0365098
:109B2800D8B499EF4DF09BEF4DF093EF4DF09DEFCA
:109B38004DF03750010D000EF324D96E030EF420BA
:109B4800DA6EDF50136E372A3F0E3764AEEF4DF0F2
:109B5800B0EF4DF0B4EF4DF0000E376EB4EF4DF0AE
:109B6800A39A3606A38A1350BAEF4DF01200090ED5
:109B78009AEC4FF0DDEC50F00001A66F080E9AEC5D
:109B88004FF0DDEC50F00001A76F060E9AEC4FF095
:109B9800DDEC50F00001A86F050E9AEC4FF0DDECFB
:109BA80050F00001A96F040E9AEC4FF0DDEC50F074
:109BB8000001AA6F030E9AEC4FF07F0BDDEC50F01A
:109BC8000001AB6F1200F5EF4DF014C0F6FF15C0A1
:109BD800F7FF0800F550DCEC4BF0144A152AF5EFB6
:109BE8004DF014C0F6FF15C0F7FF0800F550000946
:109BF800D8A401EF4EF003EF4EF0E9EF4DF005EF7A
:109C08004EF01604D8A40BEF4EF00DEF4EF011EF06
:109C18004EF010EC51F011EF4EF012000C0E4A60AD
:109C280018EF4EF01AEF4EF034EF4EF03F50010DA2
:109C3800780EF324D96E000EF420DA6EDF50AE6E83
:109C48003F2A0B0E3F642BEF4EF02DEF4EF031EF15
:109C58004EF0000E3F6E31EF4EF04A2A37EF4EF0CD
:109C68009D9837EF4EF01200400E49603EEF4EF0DF
:109C780040EF4EF05AEF4EF03950010D400EF324EC
:109C8800D96E030EF420DA6EDF50A96E392A3F0E22
:109C9800396451EF4EF053EF4EF057EF4EF0000E8F
:109CA800396E57EF4EF0492A5DEF4EF0A3985DEFFD
:109CB8004EF01200176E1450186E13C019F019C028
:109CC800F6FF18C0F7FF17C0F8FF000EA66E15C004
:109CD800F5FF0D001650F56E0C00A68AA684F29EBC
:109CE800F29C550EA76EAA0EA76EA682A694A69AF7
:109CF800F28EF28C000EA66E000EF86E1200ACA268
:109D080088EF4EF08AEF4EF08EEF4EF0AC98AC88AC
:109D18008EEF4EF03E50010D6C0EF324D96E000EFE
:109D2800F420DA6EAFCFDFFF3E2A0B0E3E649FEFC2
:109D38004EF0A1EF4EF0A5EF4EF0000E3E6EA5EFEF
:109D48004EF03C2A12009CA2ACEF4EF0AEEF4EF063
:109D5800B2EF4EF09C989C88B2EF4EF03850010D4F
:109D6800000EF324D96E030EF420DA6EAACFDFFFBB
:109D7800382A3F0E3864C3EF4EF0C5EF4EF0C9EFF6
:109D88004EF0000E386EC9EF4EF0362A12001FC092
:109D980014F020C015F00BEC4FF021502AEC4FF0D6
:109DA800226E22380F0B300FA7EC4BF021502AEC13
:109DB8004FF00F0B300FA7EC4BF0FF0EA7EC4BF05A
:109DC800FF0EA7EC4BF0FF0EA7EC4BF01200000EB5
:109DD800356E000E346E000E336E000E326E000EBD
:109DE800316E000E306E2C682D682D9EC3EC50F03D
:109DF80066EC50F020EC50F032EC51F0F6EC50F0FC
:109E080096EC50F093EC49F035EC51F0120019EF54
:109E18004FF014C0F6FF15C0F7FF0800F550A7EC87
:109E28004BF0144A152A19EF4FF014C0F6FF15C06D
:109E3800F7FF0800F5500009D8A425EF4FF027EFE9
:109E48004FF00DEF4FF029EF4FF012001E6E1EC0BD
:109E580013F0146A000E166E0A0E156E61EC46F0C9
:109E680013C01BF014C01CF01EC013F0146A000EBF
:109E7800166E0A0E156E7BEC45F01338F00B1B10AE
:109E88001D6E1D5048EF4FF01200136E3B50D8A4C2
:109E980050EF4FF052EF4FF064EF4FF01304D8A497
:109EA80058EF4FF05AEF4FF05EEF4FF00C0EBA6ECE
:109EB80064EF4FF0000EBA6E64EF4FF064EF4FF0AE
:109EC8001200000E446E77EF4FF0442A0A0E441831
:109ED800D8A471EF4FF073EF4FF077EF4FF07EEFAC
:109EE8004FF07EEF4FF09EA67CEF4FF07EEF4FF0E5
:109EF80069EF4FF09E961200156E000EA66E145074
:109F0800C00BF66E13C0F7FF15C0F8FFA684A6882D
:109F1800F29EF29C550EA76EAA0EA76EA682F28E2E
:109F2800F28C000EA66E000EF86E1200146E2AEC6B
:109F380051F0D00E17EC51F0145017EC51F02EECF4
:109F480051F0D10E17EC51F0D3EC4CF0156E1DEC1E
:109F580051F026EC51F01550B2EF4FF01200156E8B
:109F68001450176E13C018F018C0F6FF17C0F7FF8B
:109F780015C0F8FF000EA66E0900F5CF16F0000E0A
:109F8800A66E000EF86E1650CAEF4FF01200050EBE
:109F98000E01DA6F130EF66FA89CA88AA898A884F9
:109FA8009C8E9C9C9C887C86100EAB6EA49AA38A7F
:109FB800A498A388A58AA5881200E70E0F01486F08
:109FC8000B0E496FC28CC29EC280C18EC19CC1500B
:109FD800C70B2009C16EC150F80B0409C16E9E9CC5
:109FE8009D8C9F9C1200166E8994FBEF4FF084B0F5
:109FF80000EF50F002EF50F0FBEF4FF004EF50F09D
:10A00800165031EC4DF0155031EC4DF089841200AA
:10A018001BC013F01CC014F0156A8E0E166E000ECD
:10A02800176E4CEC44F013C01BF014C01CF015C0A4
:10A038001DF01FEF50F01200000E0001B56F000E6A
:10A04800B46F000EB36F000EB26F000EAF6F000E4C
:10A05800AE6F0A0E4C6E010E4B6E1200156E89948F
:10A0680036EF50F084B03BEF50F03DEF50F036EF54
:10A0780050F03FEF50F0155031EC4DF0898412004C
:10A08800AD9CAD8AAD98AD84AC8EAC9CAC887E8618
:10A09800100EB06E9E9A9D8A9E989D889F8A9F8872
:10A0A8001200206E2AEC51F0D00E17EC51F020501F
:10A0B80017EC51F01F5017EC51F01DEC51F026EC45
:10A0C80051F01200000E446E000E0001A66F000E43
:10A0D800A76F000EA86F000EA96F000EAA6F000EE2
:10A0E800AB6F12000E01FF910E0ECE6FC00ECB6E3D
:10A0F800600EBB6ECA84CA50FC0B0109CA6E000E02
:10A10800BA6E1200899E9F0E5FEC4DF042EC4CF047
:10A118000001BA6F91EC4AF013C0ACF014C0ADF076
:10A12800898E1200000E406E000E3F6E0C0E4A6EB5
:10A13800000E3E6E000E3D6E000E3C6E000E416E2F
:10A14800120013C0D9FF14C0DAFF28C0DFFF20EEC9
:10A1580001F01350D9261450DA2229C0DFFF12006B
:10A1680013C0D9FF14C0DAFF26C0DFFF20EE01F0CC
:10A178001350D9261450DA2226C0DFFF1200000E31
:10A188003A6E000E396E400E496E000E386E000EA3
:10A19800376E000E366E1200B10ED76EE00ED66E18
:10A1A800D59CD59AD598D586D58EF294F28AF18425
:10A1B8001200146E14500F0B136E14380F0B0A0D87
:10A1C800F35013261350E9EF50F01200728A72868A
:10A1D800729472927290000E716E739E739C090E47
:10A1E800746E1200000E0001BA6F000EAD6F000E03
:10A1F800AC6F000E426E12003031323334353637D0
:10A208003839414243444546136EC30EC2161344BF
:10A21800E846FC0BC21212000A0EDCEC4BF00D0EE5
:10A22800DCEC4BF01200136E13C075FF65EC4FF0B9
:10A238001200718A718865EC4FF0120060606060EE
:10A2480060606060718465EC4FF01200718065ECAD
:10A258004FF01200718265EC4FF01200000E436E51
:0EA268001200000E3B6E1200C28212001200A5
:10EB4A0000476F6C64466973682056312E31207015
:10EB5A006F776572656420757020696E205458203D
:10EB6A006D6F64652100466C617368207465737407
:10EB7A00696E67207061747465726E3A2000446928
:10EB8A0073706C617920696E207570646174652098
:10EB9A006D6F646521004343313130312052582072
:10EBAA0053796E633A2066616C73650052616469D9
:10EBBA006F207265676973746572206D61703A209F
:10EBCA0000446973706C617920696E2061707020ED
:10EBDA006D6F6465210054656D706572617475723C
:10EBEA0065205772697474656E2E00576174657278
:10EBFA00206C6576656C205772697474656E2E0098
:10EC0A004343313130312052582053796E633A20D0
:10EC1A00747275650057726974696E6720726567E8
:10EC2A006973746572732E2E2E005265736574743F
:10EC3A00696E67204343313130312E2E2E005772D0
:10EC4A006974696E67205041205461626C652E2E8A
:10EC5A002E004D455F54656D7065726174757265FD
:10EC6A002E76616C3D004C454420537472697020C5
:10EC7A005772697474656E2E004D455F57617465ED
:10EC8A00724C6576656C2E76616C3D005453545F08
:10EC9A00486F7572676C6173732E7478743D004D9A
:10ECAA00616E7566616374757265722049443A20B3
:10ECBA0000526164696F204D415243535441544597
:10ECCA003A200044524F2054656D70657261747524
:10ECDA0072653A200044524F205761746572206C65
:10ECEA006576656C3A2000537769746368657320AA
:10ECFA005772697474656E2E00526164696F205090
:10ED0A0041207461626C653A20004C6F6164696EDF
:10ED1A006720666C6173682E2E2E004572617369D6
:10ED2A006E6720666C6173682E2E2E004C696768C8
:10ED3A00747331205772697474656E2E005375703E
:10ED4A00706C7931205772697474656E2E004C6943
:10ED5A006768747332205772697474656E2E005333
:10ED6A007570706C7932205772697474656E2E00F2
:10ED7A004C696768747333205772697474656E2EB0
:10ED8A0000537570706C7933205772697474656EAC
:10ED9A002E00536B696D6D657220577269747465C4
:10EDAA006E2E005379737661727320577269747488
:10EDBA00656E2E00526164696F20504152544E555F
:10EDCA004D3A2000526164696F2056455253494FAB
:10EDDA004E3A200044524F204C45442053747269E5
:10EDEA00703A2000536176696E6720666C617368B9
:10EDFA002E2E2E0046696C746572205772697474DF
:10EE0A00656E2E004D455F50484C6576656C2E76D2
:10EE1A00616C3D005453545F4D656D6F72792E7469
:10EE2A0078743D0044524F204C6967687473313AD4
:10EE3A00200044524F20537570706C79313A20008B
:10EE4A0044524F204C6967687473323A2000445226
:10EE5A004F20537570706C79323A200044524F201B
:10EE6A004C6967687473333A200044524F205375D3
:10EE7A0070706C79333A200044524F20536B696D9D
:10EE8A006D65723A20004D455F4C494D5F302E76D4
:10EE9A00616C3D004D455F4C494D5F312E76616C8A
:10EEAA003D004D455F4C494D5F322E76616C3D0009
:10EEBA004D455F4C494D5F332E76616C3D004D45A3
:10EECA005F4C494D5F342E76616C3D004D455F4C79
:10EEDA00494D5F352E76616C3D004D455F4C494D7D
:10EEEA005F362E76616C3D004D455F4C494D5F376C
:10EEFA002E76616C3D004D455F4C494D5F382E764C
:10EF0A00616C3D0044524F2046696C7465723A2028
:10EF1A00004465766963652049443A200044545F99
:10EF2A0044412E7069633D0053535F48412E706916
:10EF3A00633D0044545F48412E7069633D0053535A
:10EF4A005F4D412E7069633D0044545F4D412E7000
:10EF5A0069633D0044545F4F412E7069633D00442C
:10EF6A00545F59412E7069633D0044545F44422EF8
:10EF7A007069633D0053535F48422E7069633D00D8
:10EF8A0044545F48422E7069633D0053535F4D42BB
:10EF9A002E7069633D0044545F4D422E7069633D93
:10EFAA000044545F4F422E7069633D0044545F59D8
:10EFBA00422E7069633D00446F6E652100446F6E96
:10EFCA00652E002E62636F3D00323100323200330B
:10EFDA0033003335003336003337004841004D41A2
:10EFEA00005041004842004D420050420050430048
:05EFFA00460053000079
:10F000000000000000000000000000000000000000
:10F0100000000000000000000000000000000000F0
:10F0200000000000000000000000000000000000E0
:10F0300000000000000000000000000000000000D0
:10F0400000000000000000000000000000000000C0
:10F0500000000000000000000000000000000000B0
:10F0600000000000000000000000000000000000A0
:10F070000000000000000000000000000000000090
:10F080000000000000000000000000000000000080
:10F090000000000000000000000000000000000070
:10F0A0000000000000000000000000000000000060
:10F0B0000000000000000000000000000000000050
:10F0C0000000000000000000000000000000000040
:10F0D0000000000000000000000000000000000030
:10F0E0000000000000000000000000000000000020
:10F0F0000000000000000000000000000000000010
:10F1000000000000000000000000000000000000FF
:10F1100000000000000000000000000000000000EF
:10F1200000000000000000000000000000000000DF
:10F1300000000000000000000000000000000000CF
:10F1400000000000000000000000000000000000BF
:10F1500000000000000000000000000000000000AF
:10F16000000000000000000000000000000000009F
:10F17000000000000000000000000000000000008F
:10F18000000000000000000000000000000000007F
:10F190000000000039300000000000000000000006
:10F1A000000000000000000000000000000000005F
:10F1B000000000000000000000000000000000004F
:06F1C00000000000000049
:08FFF800ACF302FF61F801F017
:00000001FF
